:020000040000FA
:10000000E0B50020DD010000E5010000E70100008F
:10001000E9010000EB010000ED010000000000001C
:10002000000000000000000000000000EF010000E0
:10003000F101000000000000F3010000C101000018
:10004000A93800009D3A0000FB010000FD010000FE
:10005000FF01000001020000030200000502000091
:10006000F13B0000090200000B0200000D0200003D
:100070000F02000011020000130200001502000030
:10008000B914000019020000C52C00001D02000078
:100090001F020000E53D00002302000025020000D1
:1000A00027020000290200002B0200002D020000A0
:1000B0002F02000031020000330200003502000070
:1000C00037020000390200003B0200003D02000040
:1000D0003F02000041020000430200004502000010
:1000E00047020000490200004B0200004D020000E0
:1000F0004F020000510200005302000055020000B0
:1001000057020000590200005B0200005D0200007F
:100110005F0200006102000063020000650200004F
:1001200067020000690200006B0200006D0200001F
:100130006F020000710200007302000075020000EF
:1001400077020000790200007B0200007D020000BF
:100150007F0200008102000083020000850200008F
:1001600087020000890200008B0200008D0200005F
:100170008F02000091020000D114000095020000DF
:1001800097020000990200009B0200009D020000FF
:100190009F020000A1020000A3020000A5020000CF
:1001A000A7020000A9020000DFF810D000F016FF3F
:1001B00000F0CEF80048004721580000E0B50020CC
:1001C00030B410B50348804730BCAE4630BC02485E
:1001D000004770479D650000AD33000033488047FD
:1001E00033480047FEE7FEE7FEE7FEE7FEE7FEE7EF
:1001F000FEE7FEE7FEE7FEE7FEE7FEE7FEE7FEE7D7
:10020000FEE7FEE7FEE7FEE7FEE7FEE7FEE7FEE7C6
:10021000FEE7FEE7FEE7FEE7FEE7FEE7FEE7FEE7B6
:10022000FEE7FEE7FEE7FEE7FEE7FEE7FEE7FEE7A6
:10023000FEE7FEE7FEE7FEE7FEE7FEE7FEE7FEE796
:10024000FEE7FEE7FEE7FEE7FEE7FEE7FEE7FEE786
:10025000FEE7FEE7FEE7FEE7FEE7FEE7FEE7FEE776
:10026000FEE7FEE7FEE7FEE7FEE7FEE7FEE7FEE766
:10027000FEE7FEE7FEE7FEE7FEE7FEE7FEE7FEE756
:10028000FEE7FEE7FEE7FEE7FEE7FEE7FEE7FEE746
:10029000FEE7FEE7FEE7FEE7FEE7FEE7FEE7FEE736
:1002A000FEE7FEE7FEE7FEE7FEE700004D24000064
:1002B000A901000040EA01039B0703D009E008C937
:1002C000121F08C0042AFAD203E011F8013B00F81B
:1002D000013B521EF9D27047D2B201E000F8012B67
:1002E000491EFBD270470022F6E710B513460A46B6
:1002F00004461946FFF7F0FF204610BD10B5002256
:1003000000E0521C835C8C5CA34201D1002BF8D12D
:10031000D8B2E1B2401A10BD0FB400B58DB010A92B
:1003200009900B9000914FF0FF300A9000200C9044
:1003300005480690054807906A4609A80F9900F0FD
:1003400079FC0DB05DF814FB510C00006F0C00003F
:1003500070B5054C054D04E020460168084480470F
:10036000241DAC42F8D170BD748400007884000074
:100370002DE9F04D81EA030404F0004B21F0004523
:1003800014464FF0000A23F0004150EA050220D045
:1003900054EA01021DD0C5F30A570246C5F3130300
:1003A000C1F31300C1F30A5640F4801543F48013DF
:1003B000A7EB0608101BD64608F2FD3873EB0500C4
:1003C00002D308F1010801E092185B41B8F1000F77
:1003D00003DA00200146BDE8F08D00204FF48011C3
:1003E000064684460EE0171B73EB050705D3121B68
:1003F00063EB050306434CEA010C49084FEA300061
:1004000092185B4150EA0107EDD152EA030012D085
:1004100082EA040083EA0501084305D0101BAB41C2
:1004200006D20122002306E000224FF0004302E042
:100430006FF0010253101AEB06004CEB085110EB61
:100440000A0041EB0B01BDE8F04D00F021BC0EB5F8
:1004500040F2334202920022CDE90022134600F01E
:1004600026FC03B000BDC1F30A5210B5C1F313015D
:1004700040F2FF3341F480119A4201DA002010BDAE
:1004800040F233439A42A2F2334203DC524200F07C
:100490004AF810BD904010BD30B50B460146002013
:1004A0002022012409E021FA02F59D4205D303FA36
:1004B00002F5491B04FA02F52844151EA2F10102B7
:1004C000F1DC30BD2DE9F05F0546002092469B46E9
:1004D00088460646814640241BE02846414647465A
:1004E000224600F020F853465A46C01A914110D3D4
:1004F00011461846224600F083FD2D1A67EB0108CD
:100500004F4622460120002100F07AFD17EB00093A
:100510004E41201EA4F10104DFDC484631462A4644
:100520004346BDE8F09F202A04DB203A21FA02F07E
:100530000021704721FA02F3D040C2F1200291401D
:100540000843194670472DE9FF4F1C4681B0002132
:10055000D4E9016791464FF0FF358A468846A16984
:100560006D1C02988847216A834688470028F6D187
:10057000BBF1FF3F0CD026F4C066002F1ADD7006D9
:1005800015D5BBF12B0F0AD0BBF12D0F0FD104E015
:100590004FF0FF3005B0BDE8F08F46F48066A169EA
:1005A0006D1C029888477F1E8346002F02DDBBF139
:1005B000300F03D0B9F1000F2AD025E0A1696D1CDE
:1005C00046F400767F1E029888478346002F05DD9B
:1005D000BBF1780F06D0BBF1580F03D0B9F1000F73
:1005E00010D011E0B9F1000F02D0B9F1100F0BD10A
:1005F000A1696D1C26F400767F1E02988847834609
:10060000102000E0082081464FEAE970009017E0D2
:100610000A20F8E74346AAFB092803FB0980DDF816
:1006200000C07F1E0AFB0C0112EB0B0A41EBEB78BA
:10063000A16946F4007605F10105029888478346D2
:10064000002F06DD4946584600F000FD5FEA000B2A
:10065000E0D5E16902988847B00502D46FF0010047
:1006600098E7F00718D1700610D57005514605D5EA
:100670000023D1EB030163EB080200E0424620684F
:10068000031D23600068C0E9001205E02068011D19
:1006900021600068C0E900A828467BE72DE9FF5FDC
:1006A0001D464FF0FF3BD5E9014691465F464FF0AE
:1006B0000008A9697F1C01988847296A82468847F3
:1006C0000028F6D1BAF1FF3F0CD024F4C064002E0C
:1006D00019DD600614D5BAF12B0F09D0BAF12D0F30
:1006E0000ED103E0584604B0BDE8F09F44F48064A6
:1006F000A9697F1C01988847761E8246002E02DD7C
:10070000BAF1300F03D0B9F1000F26D032E0A96959
:10071000761E44F400747F1C019888478246002EA0
:1007200005DDBAF1780F06D0BAF1580F03D0B9F150
:10073000000F10D01EE0B9F1000F02D0B9F1100F78
:1007400018D1A969761E24F400747F1C019888478B
:100750008246102002E0082000E00A20814609E0DD
:1007600008FB0908A969761E44F400747F1C0198EF
:1007700088478246002E05DD4946504600F066FC5B
:100780000028EDDAE96901988847A00502D46FF0E6
:100790000100A8E7E00725D1600613D5600502D562
:1007A000C8F1000000E0404629680A1D2A60096877
:1007B000220501D5087015E0220701D5088011E057
:1007C00008600FE02868011D29600068210502D536
:1007D00080F8008006E0210702D5A0F8008001E043
:1007E000C0F8008038467EE72DE9FF5FD2E901A717
:1007F0004FF00008916999461446DDF838B0464636
:1008000001988847054659EA0B0005D009E0A1691F
:10081000761C019888470546216A284688470028A3
:10082000F5D1681C03D05FEACA7005D015E04FF01F
:10083000FF3004B0BDE8F09F2068011D2160D0F8B2
:1008400000800AE05FEACA7001D108F8015BA16983
:10085000761C7F1E019888470546002F1ADD681C0C
:1008600018D0B9F1000F0DD0E81705EBD060421198
:1008700020F01F0059F822102A1A0120904001424E
:10088000E0D107E0BBF1000FDCD1216A28468847A0
:100890000028D7D0E16901988847BBF1000F07D144
:1008A000002E05DD5FEACA7002D1002188F8001031
:1008B000A068B84203DDBBF1000F03D017B16FF0A1
:1008C0000100B6E73046B4E72DE9FF4F087883B062
:1008D0009946FF2805D0491C2D2804D0002400206B
:1008E00008E000200BE00124F9E700EB800003EBB7
:1008F0004000491C0B78FF2BF7D104B14042002384
:100900000293147819461D462D2C01D02B2C04D1AE
:10091000521C2D2C13D000240294AA461478FF2CCC
:100920000FD00A25A3FB057801FB05814FF0000CD1
:1009300003FB0C11521CE3194AEB0101EEE7012401
:10094000EAE7814453EA010002D019F5C87F06DACC
:1009500003980021C0E9001107B0BDE8F08F002521
:10096000AE4E2F46DFF8B8821846FFF770FDCDE98E
:100970000001B9F1000002DAC9F1000400E0044608
:100980000023A74A1AEB030B42EB045A12E0E007DC
:1009900007D02A4633463846414600F07DFA0746DE
:1009A00088462A4633461046194600F075FA054631
:1009B0000E466410002CEAD1DDE90001B9F1000F08
:1009C0005A46534606DAFFF7D3FC3A464346FFF74A
:1009D000CFFC05E000F060FA3A46434600F05CFACE
:1009E000029A0AB181F00041039AC2E90001B3E71B
:1009F0002DE9FF4F1F468DB0D7E901464FF0FF3874
:100A00002E2045464FF000090B90B9696D1C0E98D9
:100A10008847396A824688470028F6D1BAF1FF3FF5
:100A20000AD024F4D064002E11DDBAF12B0F08D0C7
:100A3000BAF12D0F0BD102E0404611B08DE744F41E
:100A40008064B9696D1C0E9888478246761E694697
:100A5000600501D52D2000E02B208DF8000001F16C
:100A6000010B0DF1200809E0B9696D1C0E9888474B
:100A700082460F9844F40074761E0560002E02DD55
:100A8000BAF1300FF0D00B998A453ED144F0800482
:100A900006E00F99681CA9F1010944F4007408608C
:100AA000B9696D1C761E0E98884782463028F0D0B2
:100AB0002BE00B998A4505D1200603D444F080042D
:100AC000761E18E0504605F023FF08B30DF113021F
:100AD000761EAAF1300044F40074934506D20BF858
:100AE000010B200607D5A9F1010003E0200602D47E
:100AF00009F101008146A00502D50F99681C086024
:100B0000B9696D1C0E9888478246002ED1DC53E0EF
:100B1000002E51DDBAF1650F02D0BAF1450F4BD16D
:100B2000A00549D5B9696D1C24F44074761E0E9851
:100B300088478246002E0CDD2B2804D0BAF12D0FF9
:100B400007D144F48074B9696D1C0E9888478246B9
:100B5000761EE00501D52D2100E02B2108F8011BB0
:100B6000CDF82C8021E00DF12901761E44F40074AB
:100B700088450CD2AAF1300010F0FF0088F8000080
:100B800002D10B99884509D908F1010806E0E00572
:100B900001D5244801E042F20F708146B9696D1C0D
:100BA0000E98884782460F980560002E04DD504657
:100BB00005F0AEFE0028D6D1F9690E988847FF20CF
:100BC0008BF8000088F800000020069007904B4644
:100BD0006A4608A906A8FFF777FEA00502D46FF0C1
:100BE00001002AE714F0240F0AD0E00714D1DDE950
:100BF00006123868031D3B600068C0E900120BE074
:100C0000DDE9060100F0C6FB0146E00704D13868C3
:100C1000021D3A600068016028460EE7000014409B
:100C20000000F03FF1D8FFFF026811441378016023
:100C300018467047D160044951610449116200218E
:100C40001161114600F010BA290C00004310000099
:100C5000426842B1016811F8013B23B1521EC0E95C
:100C60000012184670470121C160881E7047426813
:100C70005AB1C368016843B983688B4205D0491EE5
:100C8000521CC0E90012002070474FF0FF3070473F
:100C900010B5141E73F1000408DA401C41F1000184
:100CA00092185B411A4301D120F0010010BD2DE9DB
:100CB000F04D92469B4611B1B1FA81F202E0B0FAD2
:100CC00080F22032904600F09BF904460F4640EA3D
:100CD0000A0041EA0B0153465A46084313D0114615
:100CE00053EA010019D0C8F140025046FFF71BFC3F
:100CF00005460E4650465946424600F081F90843E3
:100D000005D0012004E020463946BDE8F08D0020E2
:100D1000054346EAE0762C4337430A986305E40A24
:100D2000A0EB08000022FD0A44EA47540A3002D52D
:100D300000200146E9E7010510196941DDE9084590
:100D400000196941BDE8F04DA2E72DE9FE4F80464C
:100D500081EA0300C00F0C46009021F0004123F00F
:100D60000045B8EB0200A94105D240462146904615
:100D70001C460B46024623F00040104347D0270D87
:100D8000C7F30A00C3F30A510290401A01904028A9
:100D90006BDAC3F3130040F4801B0098924620B135
:100DA0000023D2EB030A63EB0B0B01985946C0F109
:100DB0004002504600F024F906460D46504659467A
:100DC000019A00F02CF910EB08006141002487EA39
:100DD000115284EAE7731A4340D0009A62B3019A31
:100DE000012A4FEA075215DC001B61EB02014FF0AC
:100DF000004202EA0752CDE90042001C41F5801191
:100E000032462B46FFF753FF03B0BDE8F08F404654
:100E10002146F9E7001B61EB0201001C41F580133C
:100E200000185B412018A2F5001747EB030140EAC8
:100E3000D570B6196D4111E06D084FEA360645EAE6
:100E4000C0754FEA0752001B61EB0201001C41F51F
:100E5000801149084FEA30000019514132462B46B3
:100E600003B0BDE8F04FFFF713BF00980122400028
:100E70000023D0EB020263EBE073009821464FEAB7
:100E8000E074B8EB000061EB0401E9E783F0004394
:100E90005BE781F0004158E72DE9FE4F81EA03044A
:100EA00004F0004421F0004100944FF0000B23F0C7
:100EB000004350EA01045ED052EA03045BD0C3F35E
:100EC0000A54C1F30A552C44A4F2F3340194A0FB54
:100ED0000254C1F3130141F48011C3F3130343F42B
:100EE000801301FB024400FB034E840A970A44EA84
:100EF000815447EA8357A4FB076802958D0A05FBD6
:100F000007854FEA932C04FB0C542705029D4FEAFA
:100F1000065847EA1637B5EB08056EEB070C870E47
:100F2000920E47EA811742EA8312A7FB0201B6EB51
:100F30000B0164EB00042B0D43EA0C335E1844EB09
:100F40001C50DA465146E7FB0201C5F313044FEA91
:100F50000B3343EA14534FEA0432019C43EA06037D
:100F6000A4F10C040294009CCDE900B4FFF79FFEAD
:100F700003B0BDE8F08F00200146F9E7C1F30A5243
:100F8000C1F3130140F2FF3341F480119A4202DAB7
:100F900000200146704740F233439A42A2F23342A6
:100FA00002DC5242FFF7BFBA00F02AB830B5041E87
:100FB00071F1000404DB4FF00044404264EB010196
:100FC000141E73F1000405DB1C464FF0004352422F
:100FD00063EB0403994208BF904230BD064C074DB5
:100FE00006E0E06840F0010394E8070098471034F9
:100FF000AC42F6D3FFF7DCF85484000074840000A0
:10100000202A04DB203A00FA02F1002070479140C8
:10101000C2F1200320FA03F3194390407047202ABD
:1010200006DBCB17203A41FA02F043EAE07306E010
:1010300041FA02F3D040C2F1200291400843194620
:101040007047C0B24FF4F05100F0C0B93A2800D256
:10105000303820F02002412A01D3A2F13700884223
:1010600001D34FF0FF3070472DE9F34F8BB04FF0B5
:10107000000801F10C000C464FF0010B46460DF143
:10108000080A01906269012101989047051E2DD040
:10109000252D2CD0216A8847C0B1626901210198B1
:1010A0009047216A88470028F7D1411E626901985C
:1010B000904700E0761CA1690B988847216A884711
:1010C0000028F7D1E1690B988847DBE7A1690B9805
:1010D00088470746A84201D1761CD3E7E1690B98FF
:1010E00088477F1C02D1B8F1000F6FD046E100277E
:1010F00062693D463946019890472A2804D16269C1
:101100000121019890470125DFF88492626901214D
:1011100001989047A0F130010A290AD24F45E5DC39
:1011200007EB870100EB4107303FDFD445F01005A6
:10113000ECE7E90601D46FF000476C280AD04C2890
:1011400014D0682815D06A280DD074281CD07A28AD
:101150001AD01DE062690121019890476C2802D0E5
:1011600045F0040514E045F002050DE045F02005CA
:101170000AE06269012101989047682802D045F091
:10118000080505E045F40065626901210198904772
:10119000C4E9015765283DD019DC58287AD00CDC09
:1011A000452837D004DC252826D0412831D131E02C
:1011B00046282FD047282CD12CE05B2877D06128F7
:1011C00028D063287CD0642823D15AE0D0E06F284F
:1011D00048D008DC66281DD067281BD0692821D09C
:1011E0006E2816D127E0702845D0732868D075285E
:1011F00047D078280DD14DE0A1690B988847054666
:1012000025283FF469AFE1690B9888476D1C3FF4CE
:101210006AAFB3E023466A466FF001000B99FFF70F
:10122000E7FB9EE045F040006060A80723464FF0D2
:10123000000236D43EE0E8077FF447AF2068011D86
:1012400021600068290501D506701BE7290701D533
:10125000068017E7A90703D5F117C0E9006111E778
:1012600006600FE745F040006060A80723464FF096
:10127000080216D41EE040F60E0125EA0100606067
:1012800016E045F040006060A80723464FF00A02D0
:1012900007D40FE045F040006060A80708D523465A
:1012A00010226FF001000B99FFF74DF959E007E0AC
:1012B000234610226FF001000B99FFF7EFF950E081
:1012C0004FF000094F464B46632802D05B2806D0FA
:1012D00040E0E80601D40120A06001273AE06269FD
:1012E0000121019890475E2805D14FF001096269FC
:1012F000494601989047216939B900210A46534669
:1013000043F82120491C0829FADBB0B3216969B9E7
:10131000C11700EBD16253110AEB830122F01F02C7
:10132000821A01200B68904003430B60626901211F
:10133000019890475D28E8D1B9F1000F09D000204D
:10134000514651F82020D24341F82020401C082863
:10135000F7DB02AB224600976FF001000B99FFF715
:1013600043FA00280CDA401C08D1BBF1000F05D06D
:101370004FF0FF300DB0BDE8F08FFFE74046F9E7D2
:10138000E90701D108F1010806444FF0000B79E6A6
:10139000CCCCCC0C01F0004330B421F0004150EA39
:1013A000010206D00A0DA2F56072C1F31301002AF2
:1013B00002DC30BC00207047440F44EAC104C10085
:1013C000E01830BC00EBC25000F014B87F2801D9FF
:1013D000002208E0064A02EB5002C007127800D152
:1013E000120902F00F0201209040084070470000EF
:1013F0004E7000000029A8BF7047401C490008BF7C
:1014000020F00100704710B4B0FA80FC00FA0CF034
:1014100050EA010404BF10BC704749B1CCF120046C
:1014200021FA04F411FA0CF118BF012121430843F9
:10143000A3EB0C01CB1D4FEA00614FEA102042BF25
:10144000002010BC704700EBC35010440029A4BF1B
:1014500010BC7047401C490008BF20F0010010BCC0
:10146000704770B58C1810F8015B15F0070301D1B7
:1014700010F8013B2A1106D110F8012B03E010F8F7
:10148000016B01F8016B5B1EF9D12B0705D400231A
:10149000521E0DD401F8013BFAE710F8013BCB1ABC
:1014A000921C03E013F8015B01F8015B521EF9D5B1
:1014B000A142D8D3002070BD80B545F6EC01C2F240
:1014C000000148F20000C4F20A0000F081F880BD7B
:1014D00080B546F2F401C2F2000148F60000C4F201
:1014E0000A0000F075F880BD81B0009000990220DC
:1014F000486001B07047000081B000900099086812
:1015000040F00100086001B07047000080B58AB06B
:10151000DDF830C0CDF824C00893079206910590FD
:10152000FFE7059800F0A0FA50B9FFE748F2E42081
:10153000C0F2000005F00AF9012000F07FFFF0E79B
:101540000598069A06A9CB1D9DF81E10EC464FF093
:10155000000ECDF80CE0CCF804E0CCF8001001212E
:1015600000F09AFA0398ADF81200FFE7059800F032
:1015700083FAC8B9FFE7BDF8120002280ADBFFE7CB
:1015800048F2BD20C0F2000005F0E0F80598FFF732
:10159000ABFFFFE7012000F051FFFFE7BDF81200AD
:1015A0000130ADF81200E1E7059800F06DFA08B1DE
:1015B000FFE707E0069948F20E30C0F2000005F0A0
:1015C000C5F8FFE7059800F05FFA0AB080BD00009B
:1015D00080B58AB00990089100200390FFE7099830
:1015E00000F020F801460020C907029039B1FFE75A
:1015F000039900202029B8BF01200290FFE702983C
:10160000C00768B1FFE7099804A9019100F05AF9F1
:101610000199089803F0F2F8039801300390DEE78F
:101620000AB080BD81B000900098C06801B07047DA
:1016300080B586B00590049141F66810C2F20000B2
:101640000068800804994A68B0FBF2F04A7889780B
:1016500011440331B0FBF1F001380390059802907A
:1016600048F20001C4F20A01884208D0FFE702985C
:1016700048F60001C4F20A01884208D00FE00821B0
:10168000C4F20001086840F08050086007E00C21B7
:10169000C4F20001086840F400300860FFE70598D4
:1016A000FFF72AFF0599086820F0060008600498F3
:1016B00002780599086840EA420008600499487871
:1016C000897840EA01100599C8610498C1780398A7
:1016D00000F03F0040EA8110059988610398800975
:1016E000059948610599002088630599C8630499A4
:1016F000087A4A7A897A40EA821040EA41100599CC
:1017000008610598019048F20001C4F20A0188427C
:1017100008D0FFE7019848F60001C4F20A018842A8
:1017200011D021E00499087A4A7A897A1043084353
:1017300020B1FFE7102002F0EFFE03E0102002F0DE
:101740005FFEFFE710E00499087A4A7A897A10432D
:10175000084320B1FFE74E2002F0DEFE03E04E20FA
:1017600002F04EFEFFE7FFE706B080BD80B58CB00B
:101770000B900A910B9848F20001C4F20A018842CA
:1017800010D1FFE70020C4F20A00069009210123CE
:101790001A4601F075F906980A210422002301F087
:1017A0006FF918E00B9848F60001C4F20A0188426C
:1017B00010D1FFE78020C4F20A0005900522012322
:1017C000194601F05DF9059803220023194601F03E
:1017D00057F9FFE7FFE700208DF81C0004218DF882
:1017E0001D1003218DF81E1001218DF81F100A9A7B
:1017F00008928DF824108DF825008DF826000B989E
:1018000007A9FFF715FF0B9848F20001C4F20A017F
:1018100088421FD1FFE748F20000C4F20A0004909A
:101820004FF0FF320023194600F0F4F804986A469E
:1018300040F2FF71516040F20111116001214FF43B
:10184000917240F2FE7300F0A5F81020052102F01D
:10185000DBFE27E00B9848F60001C4F20A0188423B
:101860001FD1FFE748F60000C4F20A0003904FF0D2
:10187000FF320023194600F0CDF803986A4640F283
:10188000FF71516040F20111116001214FF491721A
:1018900040F2FE7300F07EF84E20062102F0B4FE06
:1018A000FFE7FFE70B9800F003F80CB080BD0000E5
:1018B00081B000900099086820F00100086001B034
:1018C0007047000083B0029001910298006CC0B292
:1018D000C009019908710298006CC0F38010019949
:1018E00048710298006C00F00F000199887101980E
:1018F000007908BBFFE70298406CC0000299896C30
:1019000040EA51100199086000200090FFE700981C
:101910000199897988420ED2FFE70298009900EB7D
:101920008100C06C0199009A1144C871FFE70098CA
:1019300001300090EBE728E00298406C40050299E6
:10194000896C40EA41300299C96C40EA4110029921
:10195000096D40EAD1000199086000200090FFE77E
:1019600000980199897988420ED2FFE70298009980
:1019700000EB8100406D0199009A1144C871FFE7A6
:10198000009801300090EBE7FFE7029904204860DF
:1019900003B0704710B584B08C4686460798069908
:1019A000CDF80CE0CDF808C0ADF80620ADF8043055
:1019B000ADF80210ADF800000299012000FA01F321
:1019C000039A516A99435162BDF806104901BDF866
:1019D000022041EA425109BA039A029B02EB8302B8
:1019E000C2F80013BDF804104901BDF8002041EA17
:1019F0004251C94309BA039A029B02EB8302C2F81F
:101A00008013029900FA01F20399886A10438862F0
:101A100004B010BD84B0039002910192009302992A
:101A2000012000FA01F3039A516A194351620199A6
:101A3000C90009BA039A029B02EB8302C2F80013A1
:101A400000996FEAC10109BA039A029B02EB830273
:101A5000C2F88013029900FA01F20399886A1043D0
:101A6000886204B07047000081B0009000988068E0
:101A7000C0F3800001B0704781B00090009880688A
:101A8000C0F3800001B0704781B00090009880687A
:101A9000C0F3C00001B0704785B0DDF818C0DDF8B4
:101AA00014C00490039102920193039800BBFFE7D6
:101AB0000598049908640298C0080499486402983B
:101AC00040010499886400200090FFE70098059980
:101AD00088420CD2FFE70198009A805C049901EBE0
:101AE0008201C864FFE7009801300090EEE729E02A
:101AF000059840F08000049908640298400D04990C
:101B000048640298400B049988640298400904993B
:101B1000C8640298C0000499086500200090FFE79F
:101B20000098059988420CD2FFE70198009A805CE2
:101B3000049901EB82014865FFE7009801300090AD
:101B4000EEE7FFE7049800684007002804D5FFE7A8
:101B50000499102048600BE0069820B9FFE704992B
:101B60000120486003E0049903204860FFE7FFE795
:101B700005B0704780B582B08DF80700062004F0EC
:101B8000C5FD9DF8070004F0D3FD04F0AFFD8DF80E
:101B9000060004F05BFD9DF8060002B080BD000069
:101BA00080B582B0292004F0B1FD022003F0F2F8E4
:101BB00004F09CFD8DF8070004F048FD9DF8070037
:101BC00002B080BD80B582B0262004F09FFD04F0F5
:101BD0008DFD8DF8070004F039FD9DF8070002B077
:101BE00080BD000080B582B00190282004F08EFDF9
:101BF00000208DF80300FFE79DF8030007280DDCA7
:101C0000FFE704F073FD01994A1C01920870FFE799
:101C10009DF8030001308DF80300EDE704F016FD98
:101C200002B080BD80B582B000208DF80700012091
:101C300004F06CFD04F05AFD8DF8070004F006FD79
:101C40009DF8070002B080BD80B582B000208DF8FD
:101C500006008DF80500272004F058FD04F0F6FC7E
:101C6000FFE70A2003F04CF800F086F88DF8050035
:101C70009DF80500102801D0FFE70CE09DF8060054
:101C8000411C8DF80610C92804DBFFE7FA208DF807
:101C9000070005E0E5E79DF805008DF80700FFE780
:101CA0009DF8070002B080BD80B5052004F02EFD30
:101CB00004F0CCFC80BD000080B582B001902320F0
:101CC00004F024FD00208DF80300FFE79DF80300D9
:101CD00003280DDCFFE70198411C0191007804F016
:101CE00027FDFFE79DF8030001308DF80300EDE7C5
:101CF00004F0ACFC02B080BD80B582B0019022201F
:101D000004F004FD00208DF80300FFE79DF80300B8
:101D100003280DDCFFE70198411C0191007804F0D5
:101D200007FDFFE79DF8030001308DF80300EDE7A4
:101D300004F08CFC02B080BD80B582B001902420FC
:101D400004F0E4FC00208DF80300FFE79DF8030099
:101D500003280DDCFFE70198411C0191007804F095
:101D6000E7FCFFE79DF8030001308DF80300EDE785
:101D700004F06CFC02B080BD80B582B02C2004F071
:101D8000C5FC04F0B3FC8DF8070004F05FFC9DF87F
:101D9000070002B080BD000080B584B08DF80F0050
:101DA000ADF80C100292BDF80C0008B9FFE72DE069
:101DB0003C2004F0ABFC9DF80F0004F0B9FC9DF84A
:101DC0000C0004F0B5FC9DF80D0004F0B1FC0120FE
:101DD00002F0E0FF0020ADF80600FFE7BDF80600C6
:101DE000BDF80C1088420EDAFFE704F07FFC029980
:101DF0000870029801300290FFE7BDF8060001303C
:101E0000ADF80600EAE704F021FCFFE704B080BD6E
:101E100080B582B08DF807003B2004F077FC9DF878
:101E2000070004F085FC04F061FCADF8040004F048
:101E30005DFC0146BDF8040000EB0120ADF8040094
:101E400004F004FCBDF8040002B080BD80B582B08F
:101E50008DF80700302004F059FC9DF8070004F0CD
:101E600067FC022002F096FF04F040FC8DF80600AB
:101E700004F0ECFB9DF8060002B080BD80B584B094
:101E8000FFF78EFEADF80E009DF80E00C00720B1E2
:101E9000FFE701A8FFF7A6FEFFE7BDF80E008007E9
:101EA000002801D5FFE7FFE7BDF80E004007002836
:101EB00007D5FFE748F2A730C0F2000004F046FC67
:101EC000FFE7BDF80E00C006002804D5FFE700209C
:101ED00000F04EF9FFE7BDF80E008006002804D59B
:101EE000FFE7012000F044F9FFE7BDF80E004006CF
:101EF000002804D5FFE7022000F03AF9FFE7BDF81B
:101F00000E000006002804D5FFE7032000F030F99A
:101F1000FFE704B080BD000080B582B06520FFF708
:101F200029FE8DF806009DF806009A2804D0FFE7E8
:101F3000FA208DF8070017E044F60000C2F2000016
:101F40000090FFF7D9FE00980430FFF7B5FE009827
:101F50000830FFF7F1FEFFF777FE8DF806009DF8D9
:101F600006008DF80700FFE79DF8070002B080BD6E
:101F700080B582B08DF8060000208DF805008DF840
:101F80000400352004F0C2FB9DF8060004F0D0FBED
:101F900004F05CFBFFE7052002F0B2FEFFF7ECFE69
:101FA0008DF804009DF80400102801D0FFE70CE034
:101FB0009DF80500411C8DF80510C92804DBFFE7DA
:101FC000FA208DF8070005E0E5E79DF804008DF89C
:101FD0000700FFE79DF8070002B080BD80B584B020
:101FE0008DF80F000291ADF80620392004F08EFB29
:101FF0009DF80F0004F09CFB9DF8060004F098FB90
:102000009DF8070004F094FB0020ADF80400FFE702
:10201000BDF80400BDF8061088420DDAFFE702980B
:10202000411C0291007804F083FBFFE7BDF8040037
:102030000130ADF80400EBE704F008FB04B080BD0C
:1020400080B582B08DF807000091312004F05EFB6E
:102050009DF8070004F06CFB0098411C009100788B
:1020600004F066FB0098411C0091007804F060FBCE
:102070000098411C0091007804F05AFB0098411C24
:102080000091007804F054FB04F0E0FA02B080BD47
:1020900080B582B08DF80700ADF80410322004F04E
:1020A00035FB9DF8070004F043FB9DF8040004F0A5
:1020B0003FFB9DF8050004F03BFB04F0C7FA02B0BB
:1020C00080BD000080B582B08DF807008DF8061045
:1020D000342004F01BFB9DF8070004F029FB9DF859
:1020E000060004F025FB04F0B1FA02B080BD000048
:1020F00080B582B08DF80700ADF80410332004F0ED
:1021000005FB9DF8070004F013FB9DF8040004F0A4
:102110000FFB9DF8050004F00BFB04F097FA02B0EA
:1021200080BD000080B584B045F63801C2F20001E0
:10213000019100200290FFF783FF01990298897AAC
:10214000FFF7C0FF01990298898AFFF7A1FF019963
:102150000298C98AFFF7CCFF0298FFF709FF8DF8B4
:102160000F009DF80F0003F03FFB04B080BD00009E
:1021700080B586B08DF817009DF81700FFF766FE52
:102180008DF816009DF81600C00708B1FFE7FFE7BD
:102190009DF816008007002801D5FFE7FFE79DF8AE
:1021A00016004007002855D5FFE79DF81700FFF7F8
:1021B0002FFEADF81400BDF8141048F20240C0F232
:1021C000000004F0C3FA9DF81700BDF8141044F69F
:1021D0002402C2F20002FFF7DFFDBDF81400082858
:1021E0002CD1FFE744F62400C2F2000001684268E7
:1021F00047F2C850C2F20000426001604078E32814
:102200001BD1FFE747F2D050C2F20000009047F226
:10221000C851C2F2000102F007FE009B186859681D
:102220009A68DB6804930392029101909DF817006D
:1022300001A91022FFF7D2FEFFE70AE09DF8170080
:10224000BDF8142044F62401C2F20001FFF7C6FED7
:10225000FFE7FFE79DF816000007002807D5FFE716
:1022600048F2CC30C0F2000004F070FAFFE79DF8AD
:102270001600C006002807D5FFE748F28F30C0F2ED
:10228000000004F063FAFFE79DF8160040060028FE
:1022900007D5FFE748F2E030C0F2000004F056FA3C
:1022A000FFE706B080BD000080B582B0019000203D
:1022B0008DF803000198006844F60001C4F204019F
:1022C000884210D0FFE70198006844F20001C4F290
:1022D0000401884207D0FFE7019944F60000C4F2E8
:1022E00004000860FFE70198006844F60001C4F2AA
:1022F000040188420AD1FFE70198006841F6BC1149
:10230000C2F20001086000F035FEFFE701980068A6
:1023100044F20001C4F2040188420AD1FFE70198A7
:10232000006841F6BC11C2F20001086000F0A4FD93
:10233000FFE700F05DFC8DF8030002B080BD0000F7
:1023400080B58CB000208DF81F0047F29002C0F2DB
:10235000000211685268069205910490FFE7049804
:1023600001284CDCFFE700200390FFE7049905A853
:1023700050F8210008A903F09BFD014600200190C0
:1023800039B1FFE7039900204029B8BF012001902F
:10239000FFE70198C00768B3FFE7089809990A9A10
:1023A0000B9B02F023FB089809990A9A0B9B02F0F9
:1023B000A5FB089809990A9A0B9B02F0D3FB089891
:1023C00008A90731009102F097FD0099089802F0E2
:1023D000ADFE0099089802F057FF089809990A9AEB
:1023E0000B9B02F057FB01208DF81F000398013072
:1023F0000390BBE7FFE7049801300490AFE702F0D9
:1024000063FE03F081F803F02FF99DF81F00C00769
:1024100090B1FFE700200290FFE7029802280ADC53
:10242000FFE703F061FC0A2000F008F8FFE70298DC
:1024300001300290F1E7FFE70CB080BD80B582B0BB
:102440000190019802F05CFC02B080BD4EF688510C
:10245000CEF20001086840F4700008607047000088
:1024600080B584B00290EFF3108072B603900298AA
:1024700001901E2810D0FFE7019828281AD0FFE706
:102480000198502824D0FFE7019878282ED0FFE744
:10249000019896283AD03AE048F6491040F6A171E2
:1024A0004FF6AC72C0F6113240F23143C1F2001364
:1024B00098473CE048F6492041F2A9414FF6AC72FA
:1024C000C0F6113240F23143C1F2001398472EE0BA
:1024D0004DF2493042F64A114FF6AC72C0F6113255
:1024E00040F23143C1F20013984720E041F68940A1
:1024F000C0F2010043F66B514FF6AC72C0F61132D8
:1025000040F23143C1F20013984710E0FFE746F272
:102510008950C0F2010044F674414FF6AC72C0F627
:10252000113240F23143C1F200139847FFE762B61F
:1025300004B080BD82B0019000910099012000FAA2
:1025400001F2019908689043086002B070470000EA
:1025500082B0019000910198006B0099C84000F092
:10256000010002B07047000080B586B0DDF824C0DD
:10257000DDF820C005900491039202930020C4F27C
:102580000A00019005980090B0F1402F6BD0FFE752
:10259000009844F60001C4F2000188426FD0FFE7C2
:1025A00000980021C4F20401884220D0FFE700987F
:1025B00040F60001C4F20401884224D0FFE70098ED
:1025C00041F20001C4F20401884228D0FFE70098DC
:1025D00041F60001C4F2040188422CD0FFE70098C4
:1025E00041F20001C4F20A01884230D053E00821D0
:1025F000C4F20001086840F0010008600020C4F245
:102600000A00019047E00821C4F20001086840F088
:10261000020008601020C4F20A0001903BE008218B
:10262000C4F20001086840F0040008602020C4F2F1
:102630000A0001902FE00821C4F20001086840F070
:10264000080008603020C4F20A00019023E00C2149
:10265000C4F20001086840F0010008604020C4F2A4
:102660000A00019017E00821C4F20001086840F058
:10267000100008608020C4F20A0001900BE00821DD
:10268000C4F20001086840F0200008609020C4F205
:102690000A000190FFE7019804990022012300F04D
:1026A000EFF90398012809D1FFE70499012000FA06
:1026B00001F2059948681043486008E00499012038
:1026C00000FA01F20599486890434860FFE70298D4
:1026D00001280BD1FFE70499012000FA01F20199CA
:1026E000D1F800011043C1F800010AE0049901206B
:1026F00000FA01F20199D1F800019043C1F80001FC
:10270000FFE7089801280BD1FFE70499012000FAA0
:1027100001F20199D1F800021043C1F800020AE069
:102720000499012000FA01F20199D1F800029043C6
:10273000C1F80002FFE7099801280BD1FFE70499CF
:10274000012000FA01F20199D1F800041043C1F808
:1027500000040AE00499012000FA01F20199D1F87D
:1027600000049043C1F80004FFE706B080BD0000FC
:1027700082B0019000910099012000FA01F20199C4
:1027800008681043086002B07047000080B582B04E
:1027900044F60000C2F2000001902421FDF7A3FDE1
:1027A000019940F6C010C0F6C870086040F6C0102D
:1027B000C0F2C81048606FF07F40886002B080BDF2
:1027C0007047000080B582B0684600234360036014
:1027D00041F60000C4F2040009210122FFF7C4FE03
:1027E00002B080BD80B582B0FFF7EAFF00208DF80F
:1027F000070045F62400C2F20000FFF755FDFFF781
:1028000053FA642002F07CFA48F21540C0F200004E
:1028100003F09CFFFFF706FA8DF807009DF80710FC
:1028200048F24340C0F2000003F090FF322002F073
:1028300067FAFFF7ABFFFFF76FFB8DF807009DF816
:10284000070002F0D1FFFFE7FFF7BCF9012804D130
:10285000FFE7C82002F054FA06E048F22A40C0F22E
:10286000000003F073FF00E0EEE700F005F8FFF76B
:1028700059FC02B080BD000045F63801C2F20001EB
:102880000020C861886148610861C860886048604C
:10289000086046F2E040C0F66410086042F2117031
:1028A00088820F20C88202208872704780B582B06B
:1028B000019041F66810C2F2000000680199B0FB77
:1028C000F1F000F025FD02B080BD000080B500F001
:1028D000DBFC43F69900C0F2000000F00FFD4FF45E
:1028E0007A70FFF7E3FFFFF76DFF02F07DF946F620
:1028F0008C41C2F20001086080BD000080B58EB03E
:102900006846002206924260026041F60000C4F26E
:10291000040002900321049101230893FFF724FE91
:102920000298069A089B69464A600A60042107914A
:10293000FFF71AFE049A0799089B3020C4F20A0098
:10294000039000F09DF80398049A069B114600F04E
:1029500097F8069B0799089A68464360036041F21E
:102960000000C4F204000590FFF7FEFD05980799EA
:10297000FFF7FEFE069A079908984FF496430A93CC
:102980008DF82C208DF82D208DF82E208DF83120FB
:102990008DF8322007238DF82F308DF830208DF8F8
:1029A00033108DF8340042F60000C4F204000990A0
:1029B0000AA901F073FB0898062101F047FE099867
:1029C00001F088FC0EB080BD80B500F047F918B961
:1029D000FFE7FFF753FAFFE780BD000080B584B042
:1029E0000020C4F20A00019003210F22029200236A
:1029F000039300F045F80198029A039B042100F02C
:102A00003FF84AF22001C4F20A0108682222C0F20B
:102A10000F021043086002F037F902F035F94AF26C
:102A20004001C4F20A01086820F0020008604AF27E
:102A30004402C4F20A0210684FF60063CFF6E04386
:102A40001840106010683C23C0F203031843106064
:102A5000086820F004000860FFE74AF24C00C4F266
:102A60000A00006808B9FFE7F7E74AF24001C4F23C
:102A70000A01086840F00100086004B080BD000051
:102A800084B003900291019200930298072813D812
:102A9000FFE7029881000F2000FA01F2039908680D
:102AA0009043086001980299890000FA01F20399A5
:102AB00008681043086016E002986FF01F0101EBF0
:102AC00080020F2000FA02F3039A50689843506086
:102AD0000198029A01EB820100FA01F20399486819
:102AE00010434860FFE7009858B1FFE702990120C2
:102AF00000FA01F20399D1F800031043C1F8000372
:102B00000AE00299012000FA01F20399D1F80003CA
:102B10009043C1F80003FFE704B0704780B586B06A
:102B200000200590FFE7059858BBFFE7059800EBEC
:102B3000400240F26011C2F2000101EB820051F844
:102B400022104268836841F6C010C2F2000001F012
:102B5000EBFD013080B9FFE7059800EB400140F242
:102B60006010C2F2000050F8211048F29420C0F228
:102B7000000003F0EBFDFFE7FFE70598013005904B
:102B8000D1E746F61841C2F2000101914BF6000070
:102B9000C4F20400029000F065F8019A029851799D
:102BA0009379D2794FF4616C01FB0CF1C3EB031301
:102BB00001EB83011144049146F65C51C2F200011D
:102BC00000F050F800200390FFE7039808280DDC80
:102BD000FFE70498039A46F63851C2F2000141F823
:102BE0002200FFE7039801300390EEE706B080BDB6
:102BF00080B582B000208DF8070041F6BC10C2F20B
:102C00000000006844F60001C4F2040188420AD1C1
:102C1000FFE741F20000C4F204000D21FFF798FC29
:102C20008DF80700FFE741F6BC10C2F20000006813
:102C300044F20001C4F2040188420AD1FFE741F2E4
:102C40000000C4F204000C21FFF782FC8DF807009D
:102C5000FFE79DF8070002B080BD000080B5FFF7D8
:102C6000C7FF80BD82B0019000910198C0680099B3
:102C7000088001988068C0F3C300009988700198AB
:102C80004068C0F344100099C8700198806800F053
:102C9000070101208840009908710198406800F000
:102CA0001F000099487101980068C0F385100099D1
:102CB00088710198006800F03F000099C87102B067
:102CC0007047000080B586B04BF60000C4F20400E7
:102CD00000F0BAF8E0B3FFE74BF60000C4F20400DE
:102CE000019000F0A9F8019846F61841C2F20001DF
:102CF0000291FFF7B7FF029B58799979DA791B7A2D
:102D000003F0BEFB05909DF817008DF81000BDF88C
:102D100016008DF811000598000A8DF8120005982C
:102D20008DF81300049800BA43F61431C2F2000182
:102D30004860049800BA44F2A041C2F20001486021
:102D4000049800BA41F6C011C2F200014860FFE7E2
:102D500006B080BD80B582B00190009100980078E7
:102D600001280AD1FFE74AF22001C4F20A010868EB
:102D700040F201121043086006E04AF25001C4F22A
:102D80000A0101200860FFE74FF08041086820F049
:102D90002000086000980278086840EA4210086045
:102DA0000C21C4F20001086840F40020086001987A
:102DB00000F05AF8FFE70198806A08B9FFE7FAE7E0
:102DC0000098C179007A40EA811001990860009862
:102DD0004179807940EA411001994860009A508811
:102DE0001179527901F03AFD0099097940EAC10060
:102DF00001998860009840880199C8600199012074
:102E0000886101991F2008620099487A897A40EA0E
:102E100041000199C8610099487A897A084320B134
:102E2000FFE7122001F090FB03E0122001F004FB09
:102E3000FFE702B080BD000081B000900099012042
:102E4000086201B07047000081B000900098006AED
:102E500000F0010001B0704781B00090009901209E
:102E6000486201B07047000081B0009000990020D6
:102E7000486201B07047000080B58EB068460022FD
:102E800009924260026041F20000C4F204000C2189
:102E900001230893FFF768FB089A099B6846436083
:102EA000036040F60000C4F2040002900E2103917A
:102EB000FFF75AFB02980399FFF73CFB4FF496701B
:102EC00001F01EFF02980399FFF752FC4FF04020DB
:102ED000049003210791FFF74BFC04980799089A87
:102EE000099BEC46CCF80430CCF80030FFF73CFBF3
:102EF00004980799FFF73CFC089A099B8020C4F2CC
:102F00000A00059002210691FFF7BAFD0598089B7B
:102F100004211A46FFF7B4FD0598069A099B05217E
:102F2000FFF7AEFD079A089909988DF831208DF8C2
:102F30002C008DF82D108DF82E1008228DF82F20E2
:102F40008DF830108DF832008DF833008DF8340094
:102F50008DF835008DF8360044F20000C4F204000C
:102F60000A900BA900F08CF80A9800F071F90EB0E5
:102F700080BD000080B58CB0684600220792426098
:102F8000026041F20000C4F204000D210123069307
:102F9000FFF7EAFA069A079B68464360036040F62B
:102FA0000000C4F2040002900C210391FFF7DCFA48
:102FB00002980399FFF7BEFA4FF4967001F0A0FE55
:102FC00002980399FFF7D4FB069944F60000C4F277
:102FD00000000490FFF7CCFB0498069A079B694613
:102FE0004B600B601146FFF7BFFA04980699FFF794
:102FF000BFFB069A079B9020C4F20A000590194671
:10300000FFF73EFD0598069B04211A46FFF738FDA1
:103010000598079B05210222FFF732FD06990798C4
:1030200003228DF829208DF824008DF825108DF8C5
:10303000261008228DF827208DF828108DF82A00F8
:103040008DF82B008DF82C008DF82D008DF82E00BA
:1030500044F60000C4F20400089009A900F010F83A
:10306000089800F0F5F80CB080BD000081B0009029
:103070000099086820F00800086001B0704700005F
:1030800080B588B0079006910020059004900798BD
:10309000039044F20001C4F20401884208D0FFE723
:1030A000039844F60001C4F20401884208D00FE0FE
:1030B0000821C4F20001086840F40050086007E0ED
:1030C0000821C4F20001086840F480400860FFE76E
:1030D0000798FFF7CBFF06984079082804D1FFE74F
:1030E00001200590049007E00698407918B9FFE7A1
:1030F00001200490FFE7FFE7079908684EF20802F5
:10310000CFF60172104008600698017890F801C06F
:103110008278C378890241EA0C2141EA42216FF0AA
:103120000F0202EB03121143027941EA0231059AC0
:1031300041EA4231049A41EA4271427902F00702BF
:10314000114302918079012805DBFFE70698807919
:103150000138019002E000200190FFE702980199F8
:1031600040EA81400699097A40EA415007990A6885
:10317000104340F0407008600799086820F04070E4
:103180000860079940F27F30086107990020C86005
:103190000699C8794A7A897A400140EA821040EA61
:1031A00041220799C8681043C8600798009044F20C
:1031B0000001C4F20401884208D0FFE7009844F6F9
:1031C0000001C4F20401884211D021E00699C879B7
:1031D0004A7A897A1043084320B1FFE7052001F0BD
:1031E000CBF903E0052001F043F9FFE710E0069971
:1031F000C8794A7A897A1043084320B1FFE7112041
:1032000001F0BAF903E0112001F032F9FFE7FFE71E
:1032100008B080BD80B541F6BC10C2F20000006865
:10322000002100F01FF8C0B280BD000080B582B060
:103230008DF8070041F6BC10C2F2000000689DF84E
:10324000071000F00FF88DF8060002B080BD0000F6
:1032500081B000900099086840F00800086001B053
:103260007047000082B00190009100980199486079
:10327000FFE7019880680007002801D4FFE7F8E71E
:103280000198406802B0704780B58AB02020C4F22F
:103290000A0001900222012302931146FFF7F0FB7E
:1032A0000198029A0321039100230493FFF7E8FB9E
:1032B000039904984FF4613206928DF81C008DF842
:1032C0001D008DF81E008DF81F108DF820008DF860
:1032D00021108DF822000A218DF823108DF824008A
:1032E00043F60000C4F20400059006A900F0D6FEE3
:1032F000059800F0EFFF0AB080BD000081B000909B
:10330000009845F63401C2F20001086001B0704730
:1033100080B584B0029002980138B0F1807F03D369
:10332000FFE7012003901AE0029801384EF21401E1
:10333000CEF2000108604FF0FF300721019101F04B
:10334000C9F901994EF21802CEF200020020106075
:103350004EF21002CEF2000211600390FFE70398D4
:1033600004B080BD82B0009000980138B0F1807F39
:1033700003D3FFE70120019015E04EF21002CEF2D8
:10338000000200201060009901394EF21403CEF2C1
:10339000000319604EF21801CEF200010860072107
:1033A00011600190FFE7019802B0704780B545F6C3
:1033B0003400C2F20000006838B1FFE745F634007F
:1033C000C2F2000000688047FFE780BD81B04FF087
:1033D00080400068C007F0B1FFE74AF20000C4F285
:1033E0000A000068800700280AD5FFE741F6681147
:1033F000C2F2000145F60020C0F26220086009E038
:1034000041F66811C2F2000142F60050C0F23110DC
:103410000860FFE788E04FF080400068C0F382005A
:103420000146009104286FD80099DFE801F0030BF2
:103430004048520041F66811C2F200014FF4FA40D0
:10344000086061E04AF24000C4F20A0000688007A8
:1034500000280AD5FFE741F66811C2F2000142F6E2
:103460000050C0F23110086009E041F66811C2F264
:10347000000141F60030C0F2B7000860FFE741F6F6
:103480006811C2F2000108684AF6AB22CAF6AA2205
:10349000A0FB020250080001A0EB520082004FF690
:1034A000FE70C1F6FF7000EA520008602CE041F6A1
:1034B0006811C2F200014FF40040086024E041F6B8
:1034C0006811C2F2000141F60030C0F2B700086096
:1034D0001AE041F66811C2F2000142F60050C0F253
:1034E000311008604AF20000C4F20A000068800748
:1034F000002808D5FFE741F66811C2F2000108680C
:1035000040000860FFE7FFE74FF080400068800759
:10351000002808D5FFE741F66811C2F200010868EB
:10352000C0080860FFE7FFE741F66810C2F200003C
:1035300000684DF68361C4F21B31A0FB0110800CC2
:1035400040F26C11C2F20001086001B07047000047
:1035500080B50821C4F20001086840F000700860DE
:103560009620FEF77DFF002002F05AFFFFF72EFFA6
:1035700041F66810C2F20000006840F60161C0F236
:103580002771884204D3FFE79620FEF769FF36E0F3
:1035900041F66810C2F2000000684BF20141C0F22F
:1035A000C441884204D3FFE77820FEF759FF25E0A5
:1035B00041F66810C2F20000006845F60121C0F231
:1035C0006221884204D3FFE75020FEF749FF14E050
:1035D00041F66810C2F2000000684CF28131C0F27E
:1035E000C911884204D3FFE72820FEF739FF03E022
:1035F0001E20FEF735FFFFE7FFE7FFE7FFE740F29A
:103600008021C4F20A01086820F00200086040F23C
:103610008011C4F20A01086820F00C0008607021D3
:10362000C4F20001086820F006000860086840F055
:103630000200086080BD000080B582B0019045F6B0
:103640005C00C2F20000016801310160016846F2CD
:103650006762C6F2666251FB02F39A1002EBD37204
:1036600002EB8202A1EB42010160006840B9FFE772
:1036700041F60000C4F204000921FEF75BFF07E0F9
:1036800041F60000C4F204000921FFF771F8FFE7DA
:1036900002B080BD80B582B0002001900090FFE7AD
:1036A00045F65800C2F20000006818B9FFE702F0C2
:1036B00005F85BE000200190FFE7019803284ED851
:1036C000FFE7019800EB800141F66C10C2F20000A8
:1036D00010F8210008B9FFE73DE045F65800C2F2B6
:1036E00000000368019800EB800141F66C10C2F203
:1036F000000000EB81025168C91A5160019901EB89
:10370000810100EB81004068002823DCFFE701987D
:1037100000EB800141F66C10C2F2000000EB810268
:103720005168936819445160019901EB810100EBE4
:103730008100C06868B1FFE7019800EB800141F6A5
:103740006C10C2F2000000EB8100C16810308847A5
:10375000FFE7FFE7FFE7019801300190ADE745F68D
:103760005801C2F2000100200860FFE798E700005E
:1037700080B582B0019047F2B822C2F20002106810
:10378000411C11604CF6CD41CCF6CC4100FB01F060
:103790004FEA700049F69911C1F69911884203D891
:1037A000FFE7FEF7CDFDFFE747F2B820C2F20000C9
:1037B000006845F62941CCF28F2100FB01F04FEA69
:1037C00070004BF65101C0F21E51884203D8FFE74A
:1037D00002F03AFCFFE702B080BD000080B584B083
:1037E000039045F66000C2F20000029000208DF8C0
:1037F0000700FFE79DF8070004283FDCFFE7029879
:10380000007808B9FFE730E00299086901380861DB
:10381000002829DCFFE70298007A0146009140B1B8
:10382000FFE70098012812D0FFE70098022804D093
:1038300015E002990020087015E00299CA6808692D
:103840001044086102984169806988470BE0029939
:1038500000200870029841698069884703E0029956
:1038600000200870FFE7FFE7FFE79DF80700013041
:103870008DF8070002981C300290BBE704B080BDB1
:1038800080B582B0019040F60000C4F20A0000F05A
:103890004FFD02B080BD000045F65801C2F20001A4
:1038A000086801300860704780B584B042F20000BB
:1038B000C4F20400102100F0ADFB002842D0FFE765
:1038C00042F20000C4F20400102100F091FB00203D
:1038D0000290FFE70298052833D8FFE742F2000084
:1038E000C4F2040003A900F0FFFCF0B9FFE747F2BF
:1038F000BC30C2F200000068B0F5807F07D3FFE75C
:1039000047F2BC31C2F2000100200860FFE70398D3
:1039100047F2BC33C2F200031A68511C196047F227
:10392000BC21C2F20001885406E047F2BC31C2F269
:10393000000100200860FFE7FFE7029801300290D5
:10394000C8E7FFE742F20000C4F204004FF48041F0
:1039500000F060FB002860D0FFE742F20000C4F2F4
:1039600004004FF4804100F043FBFFE742F2000007
:10397000C4F2040000F09AFC78BBFFE742F20000BA
:10398000C4F2040003A900F0AFFCF0B9FFE747F26E
:10399000BC30C2F200000068B0F5807F07D3FFE7BB
:1039A00047F2BC31C2F2000100200860FFE7039833
:1039B00047F2BC33C2F200031A68511C196047F287
:1039C000BC21C2F20001885406E047F2BC31C2F2C9
:1039D000000100200860FFE7C8E747F2BC30C2F2F0
:1039E00000000190026846F6FD00C2F2000047F2B6
:1039F000BC21C2F20001FCF75DFC0199086846F6A3
:103A00000022C2F2000210600020086046F6FC01AD
:103A1000C2F2000101200870FFE704B080BD000081
:103A200080B588B02020C4F20A0000900C21012348
:103A300002931A46FFF724F800980D210222002372
:103A40000193FFF71DF8019A02984FF4E1310491B8
:103A50008DF814208DF815208DF8162007218DF88B
:103A600019108DF81A208DF817108DF818001421F0
:103A70008DF81B108DF81C0042F20000C4F2040007
:103A8000039004A900F00AFB0198029900F000FEDF
:103A9000039800F01FFC08B080BD000080B582B024
:103AA00042F60000C4F20400102100F0B3FA00282E
:103AB00045D0FFE742F60000C4F20400102100F0F8
:103AC00097FA0020ADF80200FFE7BDF802000528D4
:103AD00034DCFFE742F60000C4F2040001A900F064
:103AE00003FCE8B9FFE746F67750C2F20000007821
:103AF000102807DBFFE746F67751C2F200010020ED
:103B00000870FFE7019846F67753C2F200031A786F
:103B1000511C197046F66751C2F20001885406E044
:103B200046F67751C2F2000100200870FFE7FFE778
:103B3000BDF802000130ADF80200C6E7FFE742F62B
:103B40000000C4F204004FF4804100F063FA002842
:103B50004CD0FFE742F60000C4F204004FF480416D
:103B600000F046FAFFE742F60000C4F2040000F05D
:103B70009DFB70BBFFE742F60000C4F2040001A900
:103B800000F0B2FBE8B9FFE746F67750C2F200005A
:103B90000078102807DBFFE746F67751C2F20001F4
:103BA00000200870FFE7019846F67753C2F2000341
:103BB0001A78511C197046F66751C2F200018854F8
:103BC00006E046F67751C2F2000100200870FFE7D8
:103BD000C9E746F67751C2F200010020087046F6A8
:103BE0006651C2F2000101200870FFE702B080BDFB
:103BF00080B584B043F20000C4F20400102100F04C
:103C000009FA002842D0FFE743F20000C4F20400A2
:103C1000102100F0EDF900200290FFE7029805283E
:103C200033D8FFE743F20000C4F2040003A900F018
:103C30005BFBF0B9FFE747F2C040C2F2000000684A
:103C4000B0F5807F07D3FFE747F2C041C2F2000121
:103C500000200860FFE7039847F2C043C2F2000368
:103C60001A68511C196047F2C031C2F20001885431
:103C700006E047F2C041C2F2000100200860FFE701
:103C8000FFE7029801300290C8E7FFE743F2000027
:103C9000C4F204004FF4804100F0BCF9002860D069
:103CA000FFE743F20000C4F204004FF4804100F04B
:103CB0009FF9FFE743F20000C4F2040000F0F6FAB7
:103CC00078BBFFE743F20000C4F2040003A900F050
:103CD0000BFBF0B9FFE747F2C040C2F200000068FA
:103CE000B0F5807F07D3FFE747F2C041C2F2000181
:103CF00000200860FFE7039847F2C043C2F20003C8
:103D00001A68511C196047F2C031C2F20001885490
:103D100006E047F2C041C2F2000100200860FFE760
:103D2000C8E747F2C040C2F200000190026846F6C0
:103D30000520C2F2000047F2C031C2F20001FCF7D8
:103D4000B9FA0199086846F60832C2F2000210601A
:103D50000020086046F60421C2F20001012008702C
:103D6000FFE704B080BD000080B588B02020C4F219
:103D70000A0000900222012302931946FEF780FEFA
:103D80000098029A002301931946FEF779FE019AE2
:103D900002984FF4E13104918DF814208DF815202C
:103DA0008DF8162007218DF819108DF81A208DF83E
:103DB00017108DF8180014218DF81B108DF81C00B9
:103DC00043F20000C4F20400039004A900F066F975
:103DD0000820032100F05CFC039800F07BFA08B097
:103DE00080BD000080B584B043F60000C4F204003A
:103DF000102100F00FF9002842D0FFE743F6000041
:103E0000C4F20400102100F0F3F800200290FFE754
:103E10000298052833D8FFE743F60000C4F20400F7
:103E200003A900F061FAF0B9FFE747F2C450C2F20B
:103E300000000068B0F5807F07D3FFE747F2C45168
:103E4000C2F2000100200860FFE7039847F2C45364
:103E5000C2F200031A68511C196047F2C441C2F251
:103E60000001885406E047F2C451C2F2000100206C
:103E70000860FFE7FFE7029801300290C8E76CE0B6
:103E800043F60000C4F204004FF4804100F0C2F891
:103E9000002860D0FFE743F60000C4F204004FF4AE
:103EA000804100F0A5F8FFE743F60000C4F20400EB
:103EB00000F0FCF978BBFFE743F60000C4F2040011
:103EC00003A900F011FAF0B9FFE747F2C450C2F2BB
:103ED00000000068B0F5807F07D3FFE747F2C451C8
:103EE000C2F2000100200860FFE7039847F2C453C4
:103EF000C2F200031A68511C196047F2C441C2F2B1
:103F00000001885406E047F2C451C2F200010020CB
:103F10000860FFE7C8E747F2C450C2F20000019012
:103F2000026846F60D30C2F2000047F2C441C2F208
:103F30000001FCF7BFF90199086846F61042C2F289
:103F4000000210600020086046F60C31C2F2000149
:103F50000120087000E0FFE7FFE704B080BD00002B
:103F600080B588B02020C4F20A000090022201230C
:103F700002931146FEF784FD0098029A0321002364
:103F80000193FEF77DFD019A02984FF4E13104910F
:103F90008DF814208DF815208DF8162007218DF846
:103FA00019108DF81A208DF817108DF818001421AB
:103FB0008DF81B108DF81C0043F60000C4F20400BD
:103FC000039004A900F06AF81520042100F060FBBA
:103FD000039800F07FF908B080BD000081B0009028
:103FE0000099486820F40070486001B070470000F4
:103FF00082B0019000919DF801004006002806D58E
:10400000FFE70199C86940F40050C861FFE702B0BA
:104010007047000084B0039002919DF80800C0062C
:10402000002808D5FFE7039881680120490200298C
:1040300001902DD4FFE79DF809004006002808D51F
:10404000FFE70398816801208902002901901FD4AD
:10405000FFE79DF808004007002808D5FFE7039810
:104060008168012089030029019011D4FFE7002015
:104070009DF8081049060029009006D5FFE703982F
:104080008068C0F3C0600090FFE700980190FFE7F0
:10409000019800F0010004B07047000080B584B0C2
:1040A000039002910398019042F20001C4F20401CE
:1040B000884218D0FFE7019842F60001C4F20401DB
:1040C000884218D0FFE7019843F20001C4F20401CE
:1040D000884218D0FFE7019843F60001C4F20401BA
:1040E000884218D01FE00821C4F20001086840F09F
:1040F0004000086017E00821C4F20001086840F0A1
:10410000800008600FE00821C4F20001086840F454
:104110008070086007E00821C4F20001086840F4DC
:1041200000700860FFE70398FFF758FF039988685D
:104130004CF20002C0F6FF721040886041F6681031
:10414000C2F20000006802990968B0FBF1F0421E5B
:104150000399886840EA321088600399486820F41F
:104160007C004860029908794A798979800440EA9C
:10417000C24040EA8152039948681043486003995D
:10418000C86880B2C8600299C879497A000440EAD8
:1041900001620399C8681043C8600399C86940F672
:1041A000FF729043C8610298C07A0399CA691043AC
:1041B00040F48050C8610399486844F21402904367
:1041C00048600299087A8A7A097B000140EA8200F5
:1041D00040EA813203994868104348600398009090
:1041E00042F20001C4F20401884218D0FFE70098AF
:1041F00042F60001C4F20401884221D0FFE7009892
:1042000043F20001C4F2040188422AD0FFE700987B
:1042100043F60001C4F20401884233D043E002991E
:10422000087A8A7A097B1043084320B1FFE700200F
:1042300000F0BAF903E0002000F036F9FFE732E0C1
:104240000299087A8A7A097B1043084320B1FFE774
:10425000012000F0A9F903E0012000F025F9FFE7B3
:1042600021E00299087A8A7A097B1043084320B139
:10427000FFE7082000F098F903E0082000F014F9A7
:10428000FFE710E00299087A8A7A097B1043084315
:1042900020B1FFE7152000F087F903E0152000F0BA
:1042A00003F9FFE7FFE704B080BD000081B0009094
:1042B0000098406800F00801012080EAD10001B0B8
:1042C0007047000081B00090009841680120884349
:1042D00001B0704781B000900099486840F40070C8
:1042E000486001B07047000084B0029001910298CC
:1042F0000068009000986FF35F20019908609DF8B6
:1043000001004007002803D5FFE70220039002E0E8
:1043100000200390FFE7039804B0704782B001903B
:104320008DF803109DF803000199086002B07047F2
:1043300081B0009000995520086101B070470000DD
:1043400080B584B00390029101920821C4F200016B
:10435000086840F480600860039800F047F803990B
:10436000886820F4706088600399886840F48060F1
:104370008860029848B9FFE70399886820F0040034
:104380008860072000F0ACF80EE00399886840F0E0
:104390000400886002980399486003990120C8606E
:1043A000072000F019F9FFE7019848B9FFE70399E2
:1043B000886820F00200886002980399086008E08D
:1043C0000399886840F002008860019803990860AA
:1043D000FFE704B080BD000081B0009000998868BC
:1043E00040F00100886001B07047000081B000908B
:1043F0000099886820F00100886001B070470000D3
:1044000081B08DF803009DF90300002812D4FFE766
:104410009DF9031001F01F02012090404A094EF25D
:104420008011CEF2000141F82200BFF34F8FBFF39D
:104430006F8FFFE701B0704781B08DF803009DF9E1
:104440000300002812D4FFE79DF9031001F01F02BA
:10445000012090404A094EF28011CEF2000141F84D
:104460002200BFF34F8FBFF36F8FFFE701B070479C
:1044700081B08DF803009DF90300002812D4FFE7F6
:104480009DF9031001F01F02012090404A094EF2ED
:104490008011CEF2000141F82200BFF34F8FBFF32D
:1044A0006F8FFFE701B0704781B08DF803009DF971
:1044B0000300002812D4FFE79DF9031001F01F024A
:1044C000012090404A094EF28011CEF2000141F8DD
:1044D0002200BFF34F8FBFF36F8FFFE701B070472C
:1044E00081B08DF803009DF90300002812D4FFE786
:1044F0009DF9031001F01F02012090404A094EF27D
:104500008011CEF2000141F82200BFF34F8FBFF3BC
:104510006F8FFFE701B0704781B08DF803009DF900
:10452000030000280ED4FFE79DF9031001F01F02DD
:10453000012090404A094EF20011CEF2000141F8EC
:104540002200FFE701B0704781B08DF803009DF9AC
:10455000030000280ED4FFE79DF9031001F01F02AD
:10456000012090404A094EF20011CEF2000141F8BC
:104570002200FFE701B0704781B08DF803009DF97C
:10458000030000280ED4FFE79DF9031001F01F027D
:10459000012090404A094EF20011CEF2000141F88C
:1045A0002200FFE701B0704781B08DF803009DF94C
:1045B000030000280ED4FFE79DF9031001F01F024D
:1045C000012090404A094EF20011CEF2000141F85C
:1045D0002200FFE701B0704781B08DF803009DF91C
:1045E000030000280ED4FFE79DF9031001F01F021D
:1045F000012090404A094EF20011CEF2000141F82C
:104600002200FFE701B0704782B08DF807000091EB
:104610009DF9070000280AD4FFE7009840019DF9A2
:1046200007104EF20042CEF2000288540BE00098D0
:1046300040019DF8071001F00F014EF61452CEF222
:1046400000028854FFE702B07047000082B08DF886
:10465000070000919DF9070000280AD4FFE70098A1
:1046600040019DF907104EF20042CEF2000288543C
:104670000BE0009840019DF8071001F00F014EF685
:104680001452CEF200028854FFE702B070470000D7
:1046900082B08DF8070000919DF9070000280AD428
:1046A000FFE7009840019DF907104EF20042CEF25C
:1046B000000288540BE0009840019DF8071001F0BB
:1046C0000F014EF61452CEF200028854FFE702B0FA
:1046D0007047000082B08DF8070000919DF9070037
:1046E00000280AD4FFE7009840019DF907104EF218
:1046F0000042CEF2000288540BE0009840019DF881
:10470000071001F00F014EF61452CEF20002885449
:10471000FFE702B07047000080B5012000F0D2FF33
:1047200080BD00007047000085B0039302920191A4
:1047300000900098008940F2C521884213DCFFE711
:104740000098018901EB410100EB81010198029A77
:10475000039B4B610A61C860009908890130088198
:104760000020049003E04FF0FF300490FFE704982E
:1047700005B0704785B003930292019100900098B4
:104780000089C72813DCFFE70098018901EB41018C
:1047900000EB81010198029A039B4B610A61C8609A
:1047A00000990889013008810020049003E04FF04F
:1047B000FF300490FFE7049805B0704784B0029280
:1047C000019100900098008963280FDCFFE70098B2
:1047D000018900EBC1010198029A0A61C860009941
:1047E0000889013008810020039003E04FF0FF307A
:1047F0000390FFE7039804B07047000010B584B041
:1048000002900191029800F0DBFF20B1FFE7002049
:104810008DF80F001DE0DDF808E0DEF800080EEB73
:1048200000110401019BD3F800C058689A68DB6846
:104830004EF804C0CB608A6048600298D0F8000847
:1048400001F02EF80299C1F8000801208DF80F0040
:10485000FFE79DF80F0004B010BD000010B593B045
:1048600012901191109200200E9047F29800C0F221
:1048700000000090016842688368D0F80CC0D0F84E
:1048800010E044690694CDF814E0CDF810C003930D
:10489000029201918169C269036AD0F824C0D0F8FC
:1048A00028E0C46A0C94CDF82CE0CDF828C0099318
:1048B00008920791006B0D9001200F90FFE70F9871
:1048C000119988420CD2FFE70F9901A850F82110E6
:1048D0000E9808440E90FFE70F9801300F90EEE716
:1048E00010990E9808440E909DF84800800740BB30
:1048F000FFE7129845F62941CCF28F2100FB01F029
:104900004FEAB00045F62841C0F28F21884210D806
:10491000FFE7129845F62941CCF28F2100FB01F008
:104920004FEA30104DF20A71C0F2A301884208D854
:10493000FFE71198032804D3FFE70E9801300E908B
:10494000FFE712980E9A40F26D1100FB012046F627
:104950009711CFF6F57108440E9040F26D700F90EC
:10496000FFE70F98129988422ED2FFE79DF83C008E
:10497000800720BBFFE70F9845F62941CCF28F2135
:1049800000FB01F04FEAB00045F62841C0F28F214C
:10499000884210D8FFE70F9845F62941CCF28F21C5
:1049A00000FB01F04FEA30104DF20A71C0F2A30192
:1049B000884204D8FFE70E9801300E90FFE7FFE72A
:1049C0000F9801300F90CCE70E98013044F6251176
:1049D000C2F29241A0FB0121421A01EB520291085E
:1049E000C900A1EB9201401A13B010BD85B0049329
:1049F00003920291019000200090FFE700980228A6
:104A000046DCFFE70198009A48F28821C0F20001D5
:104A100051F82210884215D1FFE7009A46F624404B
:104A2000C2F2000001218154009900EB01110198AC
:104A3000029A039BDDF810C0C1F814C00B61CA6074
:104A40008860FFE70198009A48F27C21C0F20001DB
:104A500051F82210884216D1FFE7009946F624400B
:104A6000C2F2000042180121D170009900EB01113F
:104A70000198029A039BDDF810C0C1F844C00B6492
:104A8000CA638863FFE7FFE7009801300090B5E74D
:104A900005B0704785B00493039202910190002005
:104AA0000090FFE70098082825DCFFE70198009AAE
:104AB00047F6B031C0F2000151F82210884215D1FA
:104AC000FFE7009A46F69C40C2F2000001218154A3
:104AD000009900EB01110198029A039BDDF810C0C8
:104AE000C1F818C04B610A61C860FFE7FFE7009892
:104AF00001300090D6E705B07047000085B0049300
:104B000003920291019000200090FFE70098032893
:104B100025DCFFE70198009A47F66071C0F20001BA
:104B200051F82210884215D1FFE7009A47F2402041
:104B3000C2F2000001218154009900EB011101989B
:104B4000029A039BDDF810C0C1F810C0CB608A60E8
:104B50004860FFE7FFE7009801300090D6E705B016
:104B60007047000085B004930392029101900020E9
:104B70000090FFE70098022825DCFFE70198009AE3
:104B800048F22811C0F2000151F82210884215D1D4
:104B9000FFE7009A47F28420C2F20000012181540D
:104BA000009900EB01110198029A039BDDF810C0F7
:104BB000C1F810C0CB608A604860FFE7FFE700984B
:104BC00001300090D6E705B07047000081B08DF845
:104BD00003008DF802109DF803009DF80210C840F4
:104BE00000F0010001B0704782B000208DF807008E
:104BF0002420C4F20000006800909DF80000C00767
:104C000020B1FFE700208DF807000AE09DF80000C2
:104C10008007002804D5FFE701208DF80700FFE793
:104C2000FFE79DF8070002B07047000081B04EF228
:104C30001400CEF2000000684EF21801CEF200011E
:104C40000968401A00904EF60450CEF20000006849
:104C50004001002815D5FFE74EF21400CEF2000007
:104C600000680099401A10280ADBFFE74EF2140092
:104C7000CEF2000000680099084401300090FFE780
:104C8000FFE7009801B0704781B04FF080400068A6
:104C9000C00710BBFFE74FF08040006800F01C0128
:104CA0000020B0EB910F0AD0FFE74FF08040006882
:104CB00000F01C010220B0EB910F0ED1FFE70020A5
:104CC0000090FFE70098132806D8FFE700BFFFE732
:104CD000009801300090F5E70FE000200090FFE71A
:104CE000009844F61F61884206D8FFE700BFFFE73F
:104CF000009801300090F3E7FFE701B07047000033
:104D000080B586B00590059844F28041C2F200015A
:104D1000096880FB01010391029046F69840C2F2B7
:104D2000000000685B2807DBFFE746F69840C2F208
:104D300000000068009002E05A200090FFE7009811
:104D40000190029B0399019AD017D21A884101DB86
:104D5000FFE71DE0019A02990398891A60EBE2705F
:104D60000291039000F096F803460A4602990398D0
:104D7000C918504102910390FFE700F08BF80246FA
:104D8000029B0398D21A71EB000001DAFFE7F4E707
:104D900006B080BD80B586B00590059844F2844188
:104DA000C2F20001096880FB01010391029046F6FE
:104DB0009840C2F2000000685B2807DBFFE746F678
:104DC0009840C2F200000068009002E05A20009073
:104DD000FFE700980190029B0399019AD017D21A1D
:104DE000884101DBFFE71DE0019A02990398891AC7
:104DF00060EBE2700291039000F04CF803460A4623
:104E000002990398C918504102910390FFE700F0FE
:104E100041F80246029B0398D21A71EB000001DAB6
:104E2000FFE7F4E706B080BD82B0019000910198E1
:104E300001210180019A00205080019B4CF60F0255
:104E4000CCF209025A60019A9060019A1173019A9A
:104E50005073019A91730199C87302B070470000B2
:104E600080B582B0019000919DF8041043F60000D7
:104E7000C4F20400FFF752FAFFE743F60000C4F261
:104E80000400FFF71FFA08B1FFE7F6E7019802B048
:104E900080BD000080B58AB0002005900490EFF33B
:104EA0001081079107990291EFF3108172B6089172
:104EB00002990191019903910090FFE70098011D6B
:104EC0000091A8B9FFE7FFF7B1FE0146C81747F206
:104ED0002822C2F20002D2E90032C91850410491DE
:104EE0000590FFE703980990099880F31088E5E79B
:104EF000049805990AB080BD80B58EB00D900C91D4
:104F000000200B90FFE70B9847F2CC01C0F20001A4
:104F10000968884280F0D680FFE70B9947F2D000FD
:104F2000C0F2000050F831000D99884240F0C58071
:104F3000FFE74FF0FF300A9000200990FFE7099843
:104F400043F61431C2F20001098988421EDAFFE7F4
:104F5000099800EB400143F61430C2F2000000EB68
:104F60008100C0680B9901EB410240F20401C2F2DA
:104F7000000151F82210884203D1FFE709980A90F6
:104F800004E0FFE7099801300990D8E70B9947F250
:104F9000D000C0F2000000EBC10001794079401A56
:104FA000013008900A98013000283ED0FFE7002029
:104FB0000790FFE70798089988421CDAFFE70C98EA
:104FC0000B9A47F2D001C0F2000101EBC20109794E
:104FD000079A1144405C0A9901EB410343F61431EE
:104FE000C2F2000101EB830111440874FFE7079846
:104FF00001300790DEE708980690FFE7069805283D
:1050000012DCFFE70A9800EB400143F61430C2F2CD
:10501000000000EB81000699014400200874FFE7BE
:10502000069801300690E9E746E00B9800EB400255
:1050300040F20400C2F2000000EB820150F82200AE
:105040000390486889680591049000200290FFE76A
:1050500002980899884214DAFFE70C980B9A47F2F5
:10506000D001C0F2000101EBC2010979029A11449A
:10507000405C03A911440871FFE7029801300290D7
:10508000E6E708980190FFE7019805280ADCFFE7AA
:10509000019903A8014400200871FFE7019801303D
:1050A0000190F1E70399049A059B43F61430C2F28C
:1050B0000000FFF75FFBFFE7FFE7FFE70B9801301A
:1050C0000B9020E70EB080BD80B582B0002001902B
:1050D000FFE70198022826DCFFE7019946F6244005
:1050E000C2F20000405CC00750B9FFE7019946F6E4
:1050F0002440C2F200000844C078C00770B1FFE746
:10510000019800F009FD019A46F62441C2F200011F
:1051100000208854019A1144C870FFE7FFE7019806
:1051200001300190D5E702B080BD000080B588B0A5
:105130000790069100200590FFE7059847F6D431C7
:10514000C0F200010968884280F09B80FFE7059962
:1051500047F6D830C0F2000050F831000799884275
:1051600040F08A80FFE74FF0FF300490002003906A
:10517000FFE7039841F6C011C2F200010989884295
:105180001EDAFFE7039800EB400141F6C010C2F2BF
:10519000000000EB8100C068059901EB410241F27B
:1051A0004001C2F2000151F82210884203D1FFE70A
:1051B0000398049004E0FFE7039801300390D8E7D8
:1051C0000698059A47F6D831C0F2000101EBC201FA
:1051D0000A794979805CFFF7F9FC8DF80B00049897
:1051E000013078B1FFE79DF80B0000F00100049951
:1051F00001EB410241F6C011C2F2000101EB820154
:10520000087438E0059800EB400241F24001C2F218
:10521000000101EB820051F822104268836841F6D8
:10522000C010C2F2000000F095FA18BBFFE7059825
:1052300000EB400241F24001C2F2000101EB8200AA
:1052400051F822104268836841F6C010C2F2000093
:105250000090FFF769FA00990889013801909DF8DC
:105260000B0000F00100019A02EB420201EB820107
:105270000874FFE7FFE7FFE7FFE7059801300590B7
:105280005BE708B080BD000080B582B0019000915E
:1052900001980121C0F60141884209D1FFE7009839
:1052A00040798007002803D5FFE700F07DFEFFE787
:1052B00002B080BD80B58AB00990089100200790A7
:1052C000FFE70798362800F31D81FFE7079947F6A7
:1052D0007070C0F2000050F831000999884240F027
:1052E0000C81FFE74FF0FF30069000200590FFE7AC
:1052F000059841F6C011C2F20001098988421EDA00
:10530000FFE7059800EB400141F6C010C2F2000033
:1053100000EB8100C068079901EB410241F28C511A
:10532000C2F2000151F82210884203D1FFE705982C
:10533000069004E0FFE7059801300590D8E708984B
:10534000079A47F67071C0F20001029101EBC201A9
:105350000A794979805CFFF739FC014602988DF89B
:105360001310079900EBC100807938B9FFE79DF869
:10537000130000F001008DF8120015E0079947F6C0
:105380007070C0F2000000EBC100807901280AD1E2
:10539000FFE79DF8130000F00100002818BF11205E
:1053A0008DF81200FFE7FFE70698013000286CD067
:1053B000FFE7079947F67070C0F2000000EBC100EC
:1053C000807920BBFFE79DF81200012811D0FFE78C
:1053D0009DF81200D0B9FFE7069800EB400141F6B6
:1053E000C010C2F2000000EB8100007C01280DD14A
:1053F000FFE79DF81200069901EB410241F6C0114A
:10540000C2F2000101EB82010874FFE73CE007995A
:1054100047F67070C0F2000000EBC10080790128EF
:1054200031D1FFE7069800EB400141F6C010C2F20F
:10543000000000EB8100007C012824D0FFE79DF8EC
:105440001200112811D0FFE79DF81200D0B9FFE734
:10545000069800EB400141F6C010C2F2000000EBDC
:105460008100007C11280DD1FFE79DF812000699FC
:1054700001EB410241F6C011C2F2000101EB8201D1
:105480000874FFE7FFE7FFE736E0079800EB40020C
:1054900041F28C51C2F2000101EB820051F822105E
:1054A0004268836841F6C010C2F2000000F052F971
:1054B00008BBFFE7079800EB400241F28C51C2F2B3
:1054C000000101EB820051F822104268836841F626
:1054D000C010C2F200000190FFF726F90199088977
:1054E000013803909DF81200039A02EB420201EB8F
:1054F00082010874FFE7FFE7FFE7FFE70798013045
:105500000790DEE60AB080BD80B582B00020019031
:10551000FFE7019803281FDCFFE7019947F24020CD
:10552000C2F20000405CC00788B1FFE7019947F272
:105530004020C2F20000009000EB011148680B31DE
:10554000FFF7B8FE0099019A00208854FFE7FFE7B3
:10555000019801300190DCE702B080BD80B588B0D1
:105560000790069100200590FFE70598222878DC37
:10557000FFE7059948F23410C0F2000050F83100FE
:105580000799884268D1FFE74FF0FF300490002070
:105590000390FFE7039844F2A041C2F20001098999
:1055A00088421ADAFFE7039944F2A040C2F20000F1
:1055B00000EBC100C068059A41F62001C2F200016B
:1055C00051F83210884203D1FFE70398049004E0B9
:1055D000FFE7039801300390DCE70698059A48F24C
:1055E0003411C0F2000101EBC2010A794979805CF3
:1055F000FFF7ECFA8DF80B000498013068B1FFE773
:105600009DF80B0000F00100049A44F2A041C2F2A0
:10561000000101EBC20108741DE0059A41F620016A
:10562000C2F2000101EBC20051F83210426844F2AC
:10563000A040C2F200000090FFF7C0F8009908896E
:10564000013801909DF80B0000F00100019A01EB78
:10565000C2010874FFE7FFE7FFE7059801300590F6
:1056600083E708B080BD000080B582B000200190C3
:10567000FFE7019802281FDCFFE7019947F2842029
:10568000C2F20000405CC00788B1FFE7019947F211
:105690008420C2F20000009000EB011148680B3139
:1056A000FFF75CFF0099019A00208854FFE7FFE7AD
:1056B000019801300190DCE702B080BD80B5FDF7B4
:1056C00083F980BD80B588B08DF81300EFF31080AA
:1056D000059005980290EFF3108072B6069002983C
:1056E00001900198039000200090FFE70098011DB1
:1056F0000091C0B9FFE79DF81300C00728B9FFE784
:105700004FF08070FDF72EFEFFE74EF60451CEF20B
:1057100000014FF000700860FFE7039807900798BA
:1057200080F31088E2E700F0E7FE47F22821C2F29A
:1057300000010020C1E9000047F23421C2F200015B
:10574000086047F23821C2F200010860FEF7EAFF64
:1057500008B080BD86B004930392029101900020AE
:105760000090FFE7009801990989884213DAFFE762
:105770000198009901EB410100EB8100C06802999A
:10578000884203D1FFE70120059007E0FFE700987A
:1057900001300090E6E700200590FFE7059806B08D
:1057A0007047000081B000900099D1F80008D1F84E
:1057B0000418401AB0FA80F0400901B070470000A8
:1057C00081B000900099D1F80008D1F80418013098
:1057D000C21700EB526222F07F02801A401AB0FA20
:1057E00080F0400901B0704780B582B08DF80700A5
:1057F0009DF8070010B9FFE702B080BD9DF80710C3
:1058000048F2F430C0F2000000F0A0FFFFE7C8202B
:105810000090FFF775FA0098FFF772FAF7E70000BB
:1058200080B584B0FDF794FE62B6FDF74FF8012015
:10583000FFF748FF40F60000C4F20A000190002183
:10584000039145F23552C0F20602FEF779FD019848
:10585000FEF7C2FDFCF7C6FFFEF7E2F8FDF74EF8D3
:10586000FEF782FAFEF77CFB48F20000C4F20A0061
:105870004EF64801C0F201010291FBF777FF029951
:1058800048F60000C4F20A00FBF770FF00F0DAFCF3
:10589000FDF744F9FDF7FEFE039804B080BD00005B
:1058A00081B0009000980130C11700EB516121F0E8
:1058B0007F01401A01B0704780B586B00590049111
:1058C0000392059802900299088900EB80020A2051
:1058D00000EB4200488002984088039908600298D3
:1058E00000780499087002984078049948700498E8
:1058F00002300299498800F0EDF8049804300299CA
:10590000496800F0F5F8049808300299098900F018
:10591000E1F800200190FFE7019802990989884287
:1059200024DAFFE70498019A02EB820100EB4100C0
:105930000A30029902EB420201EB8201C96800F0D1
:10594000D7F80498019A02EB820100EB410102981A
:1059500002EB420200EB8200828A4A820069C1F8AF
:105960000E00FFE7019801300190D5E7049806B0DA
:1059700080BD000080B586B0059004910392059823
:1059800002900299088900EB80020A2000EB420095
:10599000488002984088039908600298007804992A
:1059A000087002984078049948700498023002996F
:1059B000498800F08FF8049804300299496800F093
:1059C00097F8049808300299098900F083F80020BC
:1059D0000190FFE7019802990989884224DAFFE7DC
:1059E0000498019A02EB820100EB41000A3002990F
:1059F00002EB420201EB8201C96800F079F80498D9
:105A0000019A02EB820100EB4101029802EB420293
:105A100000EB8200828A4A820069C1F80E00FFE72B
:105A2000019801300190D5E7049806B080BD0000D0
:105A300080B586B005900491039205980290029972
:105A40000A890A2000EBC200488002984088039926
:105A500008600298007804990870029840780499C8
:105A60004870049802300299498800F033F804988D
:105A700004300299496800F03BF804980830029914
:105A8000098900F027F800200190FFE701980299AA
:105A9000098988421ADAFFE70498019A00EBC200EC
:105AA0000A30029901EBC201C96800F021F804989C
:105AB000019A00EBC201029800EBC2000069C1F834
:105AC0000E00FFE7019801300190DFE7049806B06F
:105AD00080BD000082B00190ADF802109DF8030077
:105AE00001990870BDF802000199487002B0704732
:105AF00082B0019000919DF8030001990870BDF8F3
:105B00000200019948700098000A01998870009875
:105B10000199C87002B0704780B592B01190119A87
:105B200046F62440C2F2000000F1080112018A5832
:105B30001092119A01EB0212D2F80710D2F80B2042
:105B40000F920E9111993830090141580D91119918
:105B500000EB0111D1F80700D1F80B100C910B905C
:105B60001198C0010A900A98803009900998B0F500
:105B70009E7F04DDFFE74FF49E700990FFE70A98CF
:105B80000890FFE708980999884280F2AA80FFE709
:105B90004FF0FF30079000200690FFE7069841F68F
:105BA000C011C2F20001098988421EDAFFE7069897
:105BB00000EB400141F6C010C2F2000000EB810092
:105BC000C068089901EB410240F27011C2F2000175
:105BD00051F82210884203D1FFE70698079004E0AD
:105BE000FFE7069801300690D8E7089947F2D010F1
:105BF000C0F20000039000EBC100027941790EA8C9
:105C0000805CFEF7E3FF01460398002918BF1121CD
:105C10008DF81710089900EBC100027941790BA8A3
:105C2000805CFEF7D3FF8DF816009DF81600012862
:105C300003D1FFE70120029003E09DF817000290D6
:105C4000FFE702988DF815000798013068B1FFE76B
:105C50009DF81500079901EB410241F6C011C2F20F
:105C6000000101EB8201087436E0089800EB400265
:105C700040F27011C2F2000101EB820051F82210D3
:105C80004268836841F6C010C2F20000FFF762FD6F
:105C900008BBFFE7089800EB400240F27011C2F227
:105CA000000101EB820051F822104268836841F63E
:105CB000C010C2F200000190FEF736FD019908897C
:105CC000013804909DF81500049A02EB420201EBA2
:105CD00082010874FFE7FFE7FFE7089801300890AA
:105CE00050E712B080BD000080B584B046F6144085
:105CF000C2F20000036844F28842C2F2000202EBE2
:105D0000C30152F833200292496803910068009061
:105D100040B1FFE70098012807D0FFE7009802286C
:105D200006D008E00A20019008E00A20019005E072
:105D30000820019002E000200190FFE702980399FB
:105D4000019A00F09FF946F61441C2F2000108687A
:105D5000013045F25652C5F2555250FB02F202EBA9
:105D6000D27202EB4202801A086004B080BD0000CB
:105D700086B0049003914FF0FF3002900020019014
:105D8000FFE7019804990989884213DAFFE704982C
:105D9000019901EB410100EB8100C0680399884241
:105DA00003D1FFE70198029004E0FFE7019801307A
:105DB0000190E6E70298013010B3FFE702980090E7
:105DC000FFE70098049909890139884211DAFFE751
:105DD0000498009901EB410100EB81018869CA69CF
:105DE0000B6A4B610A61C860FFE7009801300090C0
:105DF000E7E704990889013808810020059003E04D
:105E00004FF0FF300590FFE7059806B0704700009F
:105E100086B0049003914FF0FF3002900020019073
:105E2000FFE7019804990989884213DAFFE704988B
:105E3000019901EB410100EB8100C06803998842A0
:105E400003D1FFE70198029004E0FFE701980130D9
:105E50000190E6E70298013010B3FFE70298009046
:105E6000FFE70098049909890139884211DAFFE7B0
:105E70000498009901EB410100EB81018869CA692E
:105E80000B6A4B610A61C860FFE70098013000901F
:105E9000E7E704990889013808810020059003E0AC
:105EA0004FF0FF300590FFE7059806B070470000FF
:105EB00080B584B0029001910298FFF773FC20B185
:105EC000FFE700208DF80F001FE001990298D0F83D
:105ED000042800EB021E1201DEF80430DEF808C0D0
:105EE000DEF80CE0C1F80CE0C1F808C04B60805847
:105EF00008600298D0F80408FFF7D2FC0299C1F8B4
:105F0000040801208DF80F00FFE79DF80F0004B092
:105F100080BD000086B0049003914FF0FF300290E6
:105F200000200190FFE7019804990989884211DA5D
:105F3000FFE70498019900EBC100C068039988420B
:105F400003D1FFE70198029004E0FFE701980130D8
:105F50000190E8E702980130F0B1FFE70298009065
:105F6000FFE7009804990989013988420DDAFFE7B3
:105F70000498009900EBC10148698A690A61C86008
:105F8000FFE7009801300090EBE704990889013899
:105F900008810020059003E04FF0FF300590FFE7F7
:105FA000059806B07047000080B543F61431C2F280
:105FB00000010020088144F2A041C2F200010881E2
:105FC00041F6C011C2F200010881FFE743F6143028
:105FD000C2F20000008901280CDBFFE743F6143011
:105FE000C2F20000018901EB410150F82110FFF7D6
:105FF0000FFFEBE7FFE744F2A040C2F20000008988
:1060000001280BDBFFE744F2A040C2F20000018947
:1060100000EBC1014968FFF77DFFECE7FFE741F6C0
:10602000C010C2F20000008901280CDBFFE741F636
:10603000C010C2F20000018901EB410150F82110AB
:10604000FFF796FEEBE780BD80B586B04020C0F636
:106050000130029001208DF80C008DF80E00062012
:106060008DF80F000299039A049B0598EC46CCF832
:10607000000048F20000C4F20A00FBF747FA06B03D
:1060800080BD000080B5ADF5415D8AB00DF11C0EFC
:106090000EF541530A930DF58353099303460A986D
:1060A000836041600260436880680DF11C0E0EF54C
:1060B000015112AA98471190002010900F90FFE70D
:1060C00010981299884280F0B280FFE712981099D8
:1060D000401A0E900E98B0F5AF6F04D9FFE74FF459
:1060E000AF60089002E00E980890FFE70A9A0999BD
:1060F00008980D900D980A381368B0FBF3F00C90D7
:10610000119B18890DF5805EAEF8640018685B6815
:106110000B6041F8040C0DF11C0E0EF5825004903A
:1061200000F1080101910C99126801FB02F10A319A
:106130000B910230BDF82C10FFF7CCFC0198BDF894
:106140003010FFF7C7FC0A9B04980A30119A0F9988
:106150001B6801FB03210A310C9A02FB03F2FAF7D8
:10616000A9F80D9800F1100147F2D050C2F20000DA
:1061700003900180018813A80290FFF7ABFC0298FE
:106180000399002206924A8002304988FFF7A2FC58
:10619000029803994CF60F02CCF209024A600430CF
:1061A0004968FFF7A5FC029803994CF60302CCF26C
:1061B00009028A6008308968FFF79AFC03980499FD
:1061C000069B01220792027390F80CC08DF858C00C
:1061D0004373437B8DF859308273837B8DF85A303B
:1061E000C273C07B8DF85B001398149A159BDDF881
:1061F00058C0CDF868C019931892179017A8059049
:1062000010300D9AFAF756F8059906980D9A103243
:1062100092B2FBF7E3FE0798FCF710F90D9910987E
:10622000084410900C990F9808440F9048E7109874
:106230001299401AB0FA80F040090DF5415D0AB09C
:1062400080BD000080B58AB0694609A8086048F2A0
:106250003830C0F2000048F25531C0F2000103AA04
:10626000029207ABFAF758F8029848F26F31C0F281
:106270000001FAF743F818B9FFE7012008908EE013
:1062800048F24D31C0F2000103A8FAF737F818B907
:10629000FFE70220089081E048F27B31C0F2000164
:1062A00003A8FAF72BF818B9FFE70320089074E069
:1062B00048F27F31C0F2000103A8FAF71FF818B9BD
:1062C000FFE70420089067E048F28B31C0F200013C
:1062D00003A8FAF713F818B9FFE7052008905AE069
:1062E00048F27331C0F2000103A8FAF707F818B9B1
:1062F000FFE7062008904DE048F26B31C0F2000144
:1063000003A8F9F7FBFF18B9FFE70720089040E062
:1063100048F26731C0F2000103A8F9F7EFFF18B99E
:10632000FFE70820089033E048F27731C0F200011F
:1063300003A8F9F7E3FF18B9FFE70920089026E062
:1063400048F28331C0F2000103A8F9F7D7FF18B96A
:10635000FFE70A20089019E048F28731C0F20001F7
:1063600003A8F9F7CBFF18B9FFE70B2008900CE062
:1063700048F25131C0F2000103A8F9F7BFFF18B984
:10638000FFE70C200890FFE7FFE7FFE7FFE7FFE7E5
:10639000FFE7FFE7FFE7FFE7FFE7FFE7FFE7694604
:1063A00004A8086048F24430C0F2000048F25E31B0
:1063B000C0F2000106AA05ABF9F7AEFF45F62801C9
:1063C000C2F2000100200870099A4A80089A0A71F6
:1063D000079A4A71069A8A71059ACA71049A0A72D2
:1063E000C87201224A7288724BF60000C4F204009F
:1063F0000190FCF7AFFC0198FCF72EFD0AB080BDC0
:1064000080B54AF20001C4F20A0101200860FEF7DB
:106410003BFC4FF08041086840F00100086080BDFF
:1064200080B582B00190FFF7EBFFFCF7D7FA0421AB
:10643000C4F20001012008604FF08041086820F09C
:106440001C000860086840F004000860019838B13A
:10645000FFE74FF08041086840F00200086006E066
:106460004FF08041086820F002000860FFE74FF01D
:106470008041086820F00100086002B080BD000083
:1064800080B584B08DF80F008DF80E108DF80D20BA
:10649000ADF80A309DF80F004FF4616100FB01F088
:1064A0009DF80E10C1EB011100EB81009DF80D105D
:1064B0004218BDF80A0000214FF47A73E2FB030191
:1064C0000191009000980199F9F7C1FF41EC100B80
:1064D0009FED071B53EC112B51EC100BF9F748FF04
:1064E00041EC100B51EC100BF9F7BDFF04B080BD6F
:1064F0009A9999999999B93F80B588B041F66810F1
:10650000C2F2000001684DF68362C4F21B32A1FBA7
:106510000221890C44F28442C2F200021160006838
:1065200044F6D351C1F26201A0FB0110800944F28C
:106530008041C2F200010860EFF3108005900598D9
:106540000390EFF3108072B60690039802900298C1
:10655000049000200190FFE70198011D0191D8B936
:10656000FFE7FEF797FC46F69042C2F20002009267
:10657000C2E90001FEF78EFC0099D1E90012401A31
:1065800046F69841C2F200010860FFE704980790C0
:10659000079880F31088DFE708B080BD83B04EF223
:1065A0001400CEF20000006801300290029B47F216
:1065B0002822C2F20002D2E90001C01841F1000114
:1065C000C2E90001FFE7029A47F23021C2F200015E
:1065D000086810440860086844F28042C2F2000271
:1065E000136890FBF3F00190019812680B6800FBB0
:1065F00012300860019A47F23421C2F200010868A3
:1066000010440860FFE7FFE7029A47F23C21C2F21C
:106610000001086810440860086844F28442C2F22D
:106620000002136890FBF3F00090009812680B686A
:1066300000FB12300860009A47F23821C2F20001D4
:10664000086810440860FFE703B0704780B541F662
:10665000BC10C2F20000006844F60001C4F204015C
:10666000884208D1FFE744F60000C4F2000001218F
:10667000FCF77EF8FFE741F6BC10C2F200000068AC
:1066800044F20001C4F20401884206D1FFE74FF052
:1066900040200321FCF76CF8FFE780BD80B541F690
:1066A000BC10C2F20000006844F60001C4F204010C
:1066B000884208D1FFE744F60000C4F2000001213F
:1066C000FBF738FFFFE741F6BC10C2F2000000689C
:1066D00044F20001C4F20401884206D1FFE74FF002
:1066E00040200321FBF726FFFFE780BD80B582B085
:1066F00000208DF80700FCF78DFD8DF807000220C3
:10670000FEF748FB9DF8070002B080BD80B582B05F
:106710008DF80700FFF79AFFFFF7C0FF9DF807000D
:10672000FCF784FD0A20FEF735FB02B080BD0000B7
:1067300080B582B08DF807009DF80700FCF776FD64
:106740000220FEF727FB02B080BD00000FB4054B0E
:1067500010B503A9044A029800F0E2F810BC5DF8F5
:1067600014FB0000614E00000000002002E008C899
:10677000121F08C1002AFAD170477047002001E0BB
:1067800001C1121F002AFBD1704700002DE9FF5FF5
:1067900082B00021DDE90430020DDDF840B0034392
:1067A00018D044F61050A2F2FF324243151411984B
:1067B00001281FD0A5EB0B00401C5FEA000A4FF038
:1067C00000064E4FDFF83891B046504615D5CAF155
:1067D000000413E0119801244AA3012801D16FEAB3
:1067E0000B010298119AC0E90031C0E9024206B0DB
:1067F000BDE8F09FCBF10000DFE704460021404AEE
:10680000491842EB0450CDE9001012E0E00707D030
:1068100032463B4640464946FAF73EFB80468946AB
:1068200032463B4610461946FAF736FB06460F46F7
:106830006410002CEAD1DDE90401DDE90023BAF19E
:10684000000F06DAFAF728FB42464B46FAF724FB1C
:1068500005E0F9F78DFD42464B46F9F789FD044600
:106860000E460022284BFAF7A1FB03D84FF0FF3069
:10687000014607E00022254B20463146FAF765FA2B
:10688000FAF77CFB102409E0002C0ADB0A22002323
:10689000F9F718FE039B30321A55641E50EA0102C4
:1068A000F2D1641C039AC4F111031444119A012A11
:1068B00003D0012208430DD10AE0084304D0002090
:1068C0004FF0110B119072E7A3EB0B056D1E0DE05D
:1068D0005B4504DD4FF0000205F1010504E003DA39
:1068E0004FF00002A5F10105002AECD002981199A1
:1068F000C0E90231C0E9004579E70000000014401A
:106900000000F03F300000000000F0430000E03FD6
:1069100030380A2801D2012070470020704700005B
:106920002DE9FF4F95B09B468946064600250FE2AC
:10693000252877D100242746F84A0121059400E054
:10694000044316F8013F203B01FA03F01042F7D14F
:1069500030782A2811D06FF02F033078A0F1300260
:10696000092A16D8059A44F0020402EB820203EBCE
:1069700042021044761C0590EFE759F8042B05926B
:10698000002A03DA504244F40054059044F0020413
:10699000761C30782E2816D116F8010F44F0040426
:1069A0002A280DD06FF02F023078A0F13003092B88
:1069B00009D807EB870302EB4303C718761CF3E7FC
:1069C00059F8047B761C30786C280FD006DC4C28F4
:1069D00017D068280DD06A2814D104E0742810D08C
:1069E0007A280FD10DE044F400140AE044F4801436
:1069F00001E044F440147278824202D104F580141C
:106A0000761C761C307866280BD013DC582877D09B
:106A100009DC002875D04528F6D04628F4D0472850
:106A20001AD19DE118E0632835D0642879D0652813
:106A300012D195E1702873D008DC6728F1D069285D
:106A40006FD06E280DD06F2806D1B5E073282CD0FA
:106A5000752875D0782874D05A46179990476D1CC0
:106A600075E1C4F30250022809D003280DD0D9F8EB
:106A7000001004280DD00D6009F1040967E1D9F870
:106A80000010EA17C1E90052F6E7D9F800100D80AE
:106A9000F2E70D70F0E719F8041B8DF800100020E4
:106AA0008DF80100EA46012003E059F804AB4FF0ED
:106AB000FF3061074FF0000102D40DE008F1010141
:106AC0008846B9420FDA8045F8DB1AF80810002929
:106AD000F4D108E008F1010188468142FADB1AF896
:106AE00008100029F6D105985B46A0EB080721465F
:106AF0003846179A00F094FA284400EB080507E09E
:106B00004DE029E10DE01AF8010B5A46179990471C
:106B1000B8F10108F7D25B4621463846179A13E1CF
:106B200042E00A220092C4F302524FF0000A022A05
:106B300008D059F804CB032A4FEAEC710AD00DE0D3
:106B400029E02AE009F1070121F00702F2E802C179
:106B5000914609E00FFA8CFC4FEAEC71042A03D14C
:106B60004FFA8CFC4FEAEC71002907DA0A46002143
:106B7000DCF1000C61EB02012D2202E0220504D5BC
:106B80002B228DF80420012203E0E20701D020220D
:106B9000F7E7904659E00A2102E010220DE01021AB
:106BA0004FF0000A00910BE010224FF0000A44F071
:106BB00004040827009203E008224FF0000A009224
:106BC000C4F30252022A05D059F804CB0021032A4B
:106BD00008D009E009F1070121F00702F2E802C13B
:106BE000914605E01FFA8CFC042A01D10CF0FF0C41
:106BF0004FF00008220728D5702806D0009B83F0AC
:106C0000100353EA0A0305D00EE040228DF8042059
:106C1000012208E05CEA010206D030228DF804204F
:106C20008DF8050002229046009B83F0080353EA8A
:106C30000A030AD15CEA010201D1620705D53022BC
:106C40008DF804204FF001087F1E582804D034A08E
:106C500003900EA802900DE036A0F9E75346604677
:106C6000009AF9F72FFC84460398825C0298401E34
:106C7000029002705CEA0100F0D1029806A9081A9D
:106C800000F1200A600702D524F4803400E00127D7
:106C9000574502DDA7EB0A0000E0002000EB0A01E7
:106CA000009005984144401A0590E00306D45B46E5
:106CB0002146179A059800F0B3F90544002706E02D
:106CC00001A85A46C05D179990476D1C7F1C474527
:106CD000F6DBE0030CD55B462146179A059800F0D9
:106CE0009FF9054404E030205A46179990476D1CDF
:106CF0000099481E00900029F5DC08E002980299EE
:106D00005A460078491C0291179990476D1CBAF1B8
:106D10000001AAF1010AF1DC65E100000928010087
:106D20003031323334353637383961626364656601
:106D300000000000303132333435363738394142C3
:106D4000434445460000000000F058F90544761C15
:106D5000307800287FF4ECAD19B02846BDE8F08FFC
:106D6000620700D4062709F1070222F0070CFCE8AD
:106D70000223E14603F000485FEA080C02D00FF25C
:106D8000702C0DE05FEA045C02D50FF2682C07E07E
:106D90005FEAC47C02D00FF2602C01E0AFF2700C0D
:106DA0004FF0FF3823F00043CDF850C065280CD0D9
:106DB00006DC452809D046281DD047283DD13DE0B6
:106DC000662818D067287ED138E00021112F01DB1A
:106DD000112000E0781CCDE9000106A90EA8FFF7FC
:106DE000D5FCDDE90F010E9A03910021009207F115
:106DF000010A04914DE04FF000400097CDE90110E9
:106E000006A90EA8FFF7C2FCDDE90F0203920E9B54
:106E100011990022DDF80CA00093049211B9791C9D
:106E200000EB010AB7EB0A0004D4C0F1FF3007F110
:106E3000010A0490AAEB0700019044E0012F00DA58
:106E400001270021112F01DD112000E03846CDE996
:106E5000000106A90EA8FFF799FCDDE90F010E9AC3
:106E60000391002104910092BA4621070CD40399A2
:106E7000514500DA8A46BAF1010F05DD009AAAF100
:106E80000101515C302908D0B84202DA10F1040F38
:106E900006DA0121CDE9011015E0AAF10101E9E7C7
:106EA000002805DC049901440491AAEB000102E0EA
:106EB000411C514500DD8A460499401A401C01904E
:106EC0004FF000400290200704D40198504501DBA8
:106ED000CDF8048000208DF84F0002980DF14F0787
:106EE000B0F1004F25D02B200E9002984FF00208F1
:106EF00000280CDA404202902D200E9007E00A2173
:106F00000298F9F7C9FA3031029007F8011DB8F17B
:106F10000001A8F10108F2DC02980028EFD1791EE7
:106F20000E980870307800F0200040F0450007F817
:106F3000020D12A8C01B00F107081498007800B1D8
:106F4000012000EB0A01019801EBE0710598414432
:106F5000401A401E0590E00306D45B462146179A6E
:106F6000059800F05DF805441498007818B15A4669
:106F7000179990476D1CE00324D55B462146179A6C
:106F8000059800F04DF805441CE00498002807DB44
:106F9000DDE90301884203DD0098405C179901E0B8
:106FA000179930205A469047049805F10105401C76
:106FB00004900198401E019004D12E205A46179942
:106FC00090476D1CBAF10001AAF1010ADDDC05E071
:106FD00017F8010B5A46179990476D1CB8F100013C
:106FE000A8F10108F4DC5B462146179A0598ABE648
:106FF0002D0000002B000000200000002DE9F041D2
:10700000044600251E461746880404D405E0394688
:107010002020B0476D1C641EF9D52846BDE8F081DC
:107020002DE9F041044600251E469046C80301D5CF
:10703000302700E02027880404D505E04146384683
:10704000B0476D1C641EF9D52846BDE8F081DDDD32
:10705000DDDDDCBBBBDDDDDDDDDDDDDDDDDD98883F
:10706000888888888888777777777788888885552B
:1070700055566666666666666666666888888333A1
:10708000333222222222222222222228888D00002C
:10709000EC580020F4600020000000001F000000F9
:1070A0001C0000001F0000001E0000001F00000068
:1070B0001E0000001F0000001F0000001E00000056
:1070C0001F0000001E0000001F0000001D00000047
:1070D0000310E000000100000310E00002030000C4
:1070E0000310E000040500000310E00006070000A4
:1070F0000410E000000100000410E00002030000A2
:107100000410E000040500000410E0000607000081
:107110000510E000000100000510E000020300007F
:107120000510E000040500000510E000060700005F
:107130000610E000000100000610E000020300005D
:107140000610E000040500000610E000060700003D
:107150000710E000000100000710E000020300003B
:107160000710E000040500000710E000060700001B
:107170000810E000000100000810E0000203000019
:107180000810E000040500000810E00006070000F9
:107190000910E000000100000910E00002030000F7
:1071A0000910E000040500000910E00006070000D7
:1071B0000A10E00000010000010001014000000091
:1071C000806D00208071002000720020000000000F
:1071D0000100020A000001000100010A0000000095
:1071E0000100020A000101000100010A0001000083
:1071F0000100020A000201000100010A0002000071
:107200000100020A000301000100010A000300005E
:107210000100020A000401000100010A000400004C
:107220000100020A000501000100010A000500003A
:107230000100020A000601000100010A0006000028
:107240000100020A000701000100010A0007000016
:107250000100020A010001000100010A0100000012
:107260000100020A010101000100010A0101000000
:107270000100020A010201000100010A01020000EE
:107280000100020A010301000100010A01030000DC
:107290000100020A010401000100010A01040000CA
:1072A0000100020A010501000100010A01050000B8
:1072B0000100020A010601000100010A01060000A6
:1072C0000100020A010701000100010A0107000094
:1072D0000100020A020001000100010A0200000090
:1072E0000100020A020101000100010A020100007E
:1072F0000100020A020201000100010A020200006C
:107300000100020A020301000100010A0203000059
:107310000100020A020401000100010A0204000047
:107320000100020A020501000100010A0205000035
:107330000100020A020601000100010A0206000023
:107340000100020A020701000100010A0207000011
:107350000100020A030001000100010A030000000D
:107360000100020A030101000100010A03010000FB
:107370000100020A030201000100010A03020000E9
:107380000100020A030301000100010A03030000D7
:107390000100020A030401000100010A03040000C5
:1073A0000100020A030501000100010A03050000B3
:1073B0000100020A030601000100010A03060000A1
:1073C0000100020A030701000100010A030700008F
:1073D0000100020A040001000100010A040000008B
:1073E0000100020A040101000100010A0401000079
:1073F0000100020A040201000100010A0402000067
:107400000100020A040301000100010A0403000054
:107410000100020A040401000100010A0404000042
:107420000100020A040501000100010A0405000030
:107430000100020A040601000100010A040600001E
:107440000100020A040701000100010A040700000C
:107450000100020A050001000100010A0500000008
:107460000100020A050101000100010A05010000F6
:107470000100020A050201000100010A05020000E4
:107480000100020A050301000100010A05030000D2
:107490000100020A050401000100010A05040000C0
:1074A0000100020A050501000100010A05050000AE
:1074B0000100020A050601000100010A050600009C
:1074C0000100020A050701000100010A050700008A
:1074D0000100020A060001000100010A0600000086
:1074E0000100020A060101000100010A0601000074
:1074F0000100020A060201000100010A0602000062
:107500000100020A060301000100010A060300004F
:107510000100020A060401000100010A060400003D
:107520000100020A060501000100010A060500002B
:107530000100020A060601000100010A0606000019
:107540000100020A060701000100010A0607000007
:107550000100020A070001000100010A0700000003
:107560000100020A070101000100010A07010000F1
:107570000100020A070201000100010A07020000DF
:107580000100020A070301000100010A07030000CD
:107590000100020A070401000100010A07040000BB
:1075A0000100020A070501000100010A07050000A9
:1075B0000100020A070601000100010A0706000097
:1075C0000100020A070701000100010A0707000085
:1075D0000200010A000001000200020A000000008F
:1075E0000200010A000101000200020A000100007D
:1075F0000200020A000201000200010A000200006B
:107600000200020A000301000200010A0003000058
:107610000200020A000401000200010A0004000046
:107620000200020A000501000200010A0005000034
:107630000200020A000601000200010A0006000022
:107640000200020A000701000200010A0007000010
:107650000200020A010001000200010A010000000C
:107660000200020A010101000200010A01010000FA
:107670000200020A010201000200010A01020000E8
:107680000200020A010301000200010A01030000D6
:107690000200020A010401000200010A01040000C4
:1076A0000200020A010501000200010A01050000B2
:1076B0000200020A010601000200010A01060000A0
:1076C0000200020A010701000200010A010700008E
:1076D0000200020A020001000200010A020000008A
:1076E0000200020A020101000200010A0201000078
:1076F0000200020A020201000200010A0202000066
:107700000200020A020301000200010A0203000053
:107710000200020A020401000200010A0204000041
:107720000200020A020501000200010A020500002F
:107730000200020A020601000200010A020600001D
:107740000200020A020701000200010A020700000B
:107750000200020A030001000200010A0300000007
:107760000200020A030101000200010A03010000F5
:107770000200020A030201000200010A03020000E3
:107780000200020A030301000200010A03030000D1
:107790000200020A030401000200010A03040000BF
:1077A0000200020A030501000200010A03050000AD
:1077B0000200020A030601000200010A030600009B
:1077C0000200020A030701000200010A0307000089
:1077D0000200020A040001000200010A0400000085
:1077E0000200020A040101000200010A0401000073
:1077F0000200020A040201000200010A0402000061
:107800000200020A040301000200010A040300004E
:107810000200020A040401000200010A040400003C
:107820000200020A040501000200010A040500002A
:107830000200020A040601000200010A0406000018
:107840000200020A040701000200010A0407000006
:107850000200020A050001000200010A0500000002
:107860000200020A050101000200010A05010000F0
:107870000200020A050201000200010A05020000DE
:107880000200020A050301000200010A05030000CC
:107890000200020A050401000200010A05040000BA
:1078A0000200020A050501000200010A05050000A8
:1078B0000200020A050601000200010A0506000096
:1078C0000200020A050701000200010A0507000084
:1078D0000200020A060001000200010A0600000080
:1078E0000200020A060101000200010A060100006E
:1078F0000200020A060201000200010A060200005C
:107900000200020A060301000200010A0603000049
:107910000200020A060401000200010A0604000037
:107920000200020A060501000200010A0605000025
:107930000200020A060601000200010A0606000013
:107940000200020A060701000200010A0607000001
:107950000200020A070001000200010A07000000FD
:107960000200020A070101000200010A07010000EB
:107970000200020A070201000200010A07020000D9
:107980000200020A070301000200010A07030000C7
:107990000200020A070401000200010A07040000B5
:1079A0000200020A070501000200010A07050000A3
:1079B0000200020A070601000200010A0706000091
:1079C0000200020A070701000200010A070700007F
:1079D0000200020A000001000300010A000000008A
:1079E0000300020A000101000300010A0001000077
:1079F0000300020A000201000300010A0002000065
:107A00000300020A000301000300010A0003000052
:107A10000300020A000401000300010A0004000040
:107A20000300020A000501000300010A000500002E
:107A30000300020A000601000300010A000600001C
:107A40000300020A000701000300010A000700000A
:107A50000300020A010001000300010A0100000006
:107A60000300020A010101000300010A01010000F4
:107A70000300020A010201000300010A01020000E2
:107A80000300020A010301000300010A01030000D0
:107A90000300020A010401000300010A01040000BE
:107AA0000300020A010501000300010A01050000AC
:107AB0000300020A010601000300010A010600009A
:107AC0000300020A010701000300010A0107000088
:107AD0000300020A020001000300010A0200000084
:107AE0000300020A020101000300010A0201000072
:107AF0000300020A020201000300010A0202000060
:107B00000300020A020301000300010A020300004D
:107B10000300020A020401000300010A020400003B
:107B20000300020A020501000300010A0205000029
:107B30000300020A020601000300010A0206000017
:107B40000300020A020701000300010A0207000005
:107B50000300020A030001000300010A0300000001
:107B60000300020A030101000300010A03010000EF
:107B70000300020A030201000300010A03020000DD
:107B80000300020A030301000300010A03030000CB
:107B90000300020A030401000300010A03040000B9
:107BA0000300020A030501000300010A03050000A7
:107BB0001000010B2000010B5000010B6000010BB5
:107BC0007000010B8000010B9000010BA000010B65
:107BD000B000010B710000000300010A0602000062
:107BE0000300010A060300000300010A0604000066
:107BF0000300010A060500000300010A0606000052
:107C00000300010A060700000300010A0700000044
:107C10000300010A070100000300010A0702000037
:107C20000300010A070300000300010A0704000023
:107C30000300010A070500000300010A070600000F
:107C40000300010A070700000400010A0000000009
:107C50000400010A000100000400010A0002000003
:107C60000400010A000300000400010A00040000EF
:107C70000400010A000500000400010A00060000DB
:107C80000400010A000700000400010A01000000CE
:107C90000400010A010100000400010A01020000C1
:107CA0000400010A010300000400010A01040000AD
:107CB0000400010A010500000400010A0106000099
:107CC0000400010A010700000400010A020000008C
:107CD0000400010A020100000400010A020200007F
:107CE0000400010A020300000400010A020400006B
:107CF0000400010A020500000400010A0206000057
:107D00000400010A020700000400010A0300000049
:107D10000400010A030100000400010A030200003C
:107D20000400010A030300000400010A0304000028
:107D30000400010A030500000400010A0306000014
:107D40000400010A030700000400010A0400000007
:107D50000400010A040100000400010A04020000FA
:107D60000400010A040300000400010A04040000E6
:107D70000400010A040500000400010A04060000D2
:107D80000400010A040700000400010A05000000C5
:107D90000400010A050100000400010A05020000B8
:107DA0000400010A050300000400010A05040000A4
:107DB0000400010A050500000400010A0506000090
:107DC0000400010A050700000400010A0600000083
:107DD0000400010A060100000400010A0602000076
:107DE0000400010A060300000400010A0604000062
:107DF0000400010A060500000400010A060600004E
:107E00000400010A060700000400010A0700000040
:107E10000400010A070100000400010A0702000033
:107E20000400010A070300000400010A070400001F
:107E30000400010A070500000400010A070600000B
:107E40000400010A070700000500010A0000000005
:107E50000500010A000100000500010A00020000FF
:107E60000500010A000300000500010A00040000EB
:107E70000500010A000500000500010A00060000D7
:107E80000500010A000700000500010A01000000CA
:107E90000500010A010100000500010A01020000BD
:107EA0000500010A010300000500010A01040000A9
:107EB0000500010A010500000500010A0106000095
:107EC0000500010A010700000500010A0200000088
:107ED0000500010A020100000500010A020200007B
:107EE0000500010A020300000500010A0204000067
:107EF0000500010A020500000500010A0206000053
:107F00000500010A020700000500010A0300000045
:107F10000500010A030100000500010A0302000038
:107F20000500010A030300000500010A0304000024
:107F30000500010A030500000500010A0306000010
:107F40000500010A030700000800010A0000000004
:107F50000800010A000100000800010A00020000F8
:107F600041A1240231A1230121A1220211A1210159
:107F700011A121010000000011A121010001000058
:107F800011A121010002000011A121010003000044
:107F900011A121010004000011A121010005000030
:107FA00011A121010006000011A12101000700001C
:107FB00011A121010100000011A121010200010015
:107FC00011A121010201010011A121010202010000
:107FD00011A121010203010011A1210102040100EC
:107FE00011A121010205010011A1210102060100D8
:107FF00011A121010207010011A1210103000100CB
:1080000021A122020000000021A1220200010000A3
:1080100021A122020002000021A12202000300008F
:1080200021A122020004000021A12202000500007B
:1080300021A122020006000021A122020007000067
:1080400021A122020100000021A122020101000061
:1080500021A122020102000021A12202010300004D
:1080600031A123010000000031A123010001000023
:1080700031A123010002000031A12301000300000F
:1080800031A123010004000031A1230100050000FB
:1080900031A123010006000031A1230100070000E7
:1080A00031A123010100000031A1230102000100E0
:1080B00031A123010201010031A1230102020100CB
:1080C00031A123010203010031A1230102040100B7
:1080D00031A123010205010031A1230102060100A3
:1080E00031A123010207010031A123010300010096
:1080F00041A124020000000041A12402000100006F
:1081000041A124020002000041A12402000300005A
:1081100041A124020004000041A124020005000046
:1081200041A12402000600000600010A0100010C22
:108130000100010B0600010A040000000600010A0C
:10814000040100000600010A040200000600010A02
:10815000040300000600010A040400000600010AEE
:10816000040500000600010A040600000600010ADA
:10817000040700000600010A050000000600010ACD
:10818000050100005100010C020700005100010C24
:10819000030000005100010C030100005100010C1C
:1081A000030200005100010C030300005100010C08
:1081B000030400005100010C030500005100010CF4
:1081C000030600005100010C030700005100010CE0
:1081D000040000005100010C040100005100010CDA
:1081E000040200005100010C040300005100010CC6
:1081F000040400005100010C040500005100010CB2
:10820000040600005100010C040700005100010C9D
:10821000050000000100010C050100000100010C37
:10822000050200000100010C050300000100010B24
:10823000000000000100010B000100000100010B23
:10824000000200000100010B000300000100010C0E
:10825000030000000100010C030100000100010CFB
:10826000030200000100010C030300000100010CE7
:10827000030400000100010C030500000100010AD5
:108280000200010A0300010A0100020A0200020AB8
:108290000300020A4661696C656420746F206164A2
:1082A0006420416C61726D4576656E7420776974E7
:1082B000682043414E49443A2025780A0043414E04
:1082C000206D6573736167652073656E64207469E2
:1082D0006D656F75742E2041626F7274696E672EC2
:1082E0002E2E0A0057616974696E6720666F7220CE
:1082F00043414E2054582062756666657220746F43
:108300002062652072656164792E2E2E0A00466116
:10831000696C656420746F2073656E642043414E00
:10832000206D6573736167652077697468204944BF
:108330003A20307825580A004465632032302032D4
:108340003032330030303A32323A313900466562E9
:10835000004465630025732025642025640025649E
:108360003A25643A256400417567004A756C004AF5
:10837000616E004A756E00536570004D6172004178
:108380007072004F6374004E6F76004D6179005338
:10839000494E545F535441545F444953434F4E4EEA
:1083A000454354200D0A00496E697420737461744A
:1083B0007573203A2047494E545F535441545F50DF
:1083C00048595F4348414E47450D0A0053494E54B2
:1083D0005F535441545F434F4E4E4543540D0A0082
:1083E00053494E545F535441545F54494D5F4F5568
:1083F000540D0A004572726F723A20253032580DC2
:108400000A0072656365697665206C656E203D20A3
:1084100025640D0A004348333932455654205465CB
:1084200073742044656D6F0D0A0043483339322060
:10843000436F6E6E6563742045746865726E657413
:108440000D0A004348333932564552203A2025322E
:10845000780D0A0080840000000000200048000021
:1084600062140000808A000000480020E06D0000D7
:108470007C670000A5C2FFFF0000000000000000B4
:108480004185E00661309AF00C118A070C9A100CB5
:108490009A200C9A300C9A400C9A500C9A600C9AC4
:1084A000700C9A800C9A900C9AA00C9AB00C9AC0FE
:1084B0000C9AD00C9AE00C9AF00C119A08C0990C06
:1084C0009A200C9A300C9A400C9A500C9A600C9A94
:1084D000700C9A800C9A900CAAA0247B02B00C4AD3
:1084E0000C4289A0990C0A15100C0A15200C0A15CB
:1084F000300C0A15400C0A15500C0A15600C0A15B0
:10850000700C0A15800C0A15900C0A15A00C0A159F
:10851000B00C0A15C00C0A15D00C0A15E00C0A158F
:10852000F00C110A14010C0A15100C0A15200C0A83
:1085300015300C0A15400C0A15500C0A15600C0A6F
:1085400015700C0A15800C0A15900C0A15A00C0A5F
:1085500015B00C0A15C00C0A15D00C0A15E00C0A4F
:1085600015F00C110A14020C0A15100C0A15200C37
:108570000A15300C0A15400C0A15500C0A15600C2F
:108580000A15700C0A15800C0A15900C0A15A00C1F
:108590000A15B00C0A15C00C0A15D00C0A15E00C0F
:1085A0000A15F00C110A14030C0A15100C0A1520F8
:1085B0000C0A15300C0A15400C0A15500C0A1560EF
:1085C0000C0A15700C0A15800C0A15900C0A15A0DF
:1085D0000C0A15B00C0A15C00C0A15D00C0A15E0CF
:1085E0000C0A15F00C110A14040C0A15100C0A15CB
:1085F000200C0A15300C0A15400C0A15500C0A15EF
:10860000600C0A15700C0A15800C0A15900C0A15DE
:10861000A00C0A15B00C0A15C00C0A15D00C0A15CE
:10862000E00C0A15F00C110A14050C0A15100C0ABE
:1086300015200C0A15300C0A15400C0A15500C0AAE
:1086400015600C0A15700C0A15800C0A15900C0A9E
:1086500015A00C0A15B00C0A15C00C0A15D00C0A8E
:1086600015E00C0A15F00C110A14060C0A15100C72
:108670000A15200C0A15300C0A15400C0A15500C6E
:108680000A15600C0A15700C0A15800C0A15900C5E
:108690000A15A00C0A15B00C0A15C00C0A15D00C4E
:1086A0000A15E00C0A15F00C110A14070C0A151033
:1086B0000C0A15200C0A15300C0A15400C0A15502E
:1086C0000C0A15600C0A15700C0A15800C0A15901E
:1086D0000C0A15A00C0A15B00C0A15C00C0A15D00E
:1086E0000C0A15E00C0A15F00C110A14080C0A15F6
:1086F000100C0A15200C0A15300C0A15400C0A152E
:10870000500C0A15600C0A15700C0A15800C0A151D
:10871000900C0A15A00C0A15B00C0A15C00C0A150D
:10872000D00C0A15E00C0A15F00C110A14090C0AF9
:1087300015100C0A15200C0A15300C0A15400C0AED
:1087400015500C0A15600C0A15700C0A15800C0ADD
:1087500015900C0A15A00C0A15B00C0A15C00C0ACD
:1087600015D00C19B6790C9A100C9A200C9A300C72
:108770009A400C9A500C9A600C9A700C9A800C9A41
:10878000900C9AA00CAAB00C8A080C9AC0189AD027
:108790000C9AE00C9AF00C119A01CC990C9A200CCE
:1087A0009A300C9A400C9A500C9A600C9A700C9A61
:1087B000800C9A900C9AA00C9AB00C9AC00C9AD08B
:1087C0000CAAE02499F09AF018119A02CC990C9A0C
:1087D000200C9A300C9A400C9A500C9A600C9A70AB
:1087E0000C9A800C9A900C9AA00C9AB00C9AC00C1F
:1087F0009AD00C9AE00C9AF00C119A03C0990C9A3A
:10880000D0F09A20189A300C9A400C9A500C9A602A
:108810000C9A700C9A800C9A900C9AA00C9AB00C3E
:10882000AAC090990C9AE00C9AF00C119A04CC9979
:108830000C9A200C9A300C9A400C9A500C9A600CAE
:108840009A700C9A800C9A900C9AA00C9AB00C9A80
:10885000C00C9AD00C9AE00C9AF00C119A05C099B1
:108860000C9A200C9A300C9A400C9A500C9A600C7E
:108870009A700C9A800C9A900C9AA00C9AB00C9A50
:10888000C00C9AD00C9AE00C9AF00C119A06C09980
:108890000C9A200C9A300C9A400C9A500C9A600C4E
:1088A0009A700C9A800C9A900C9AA00C9AB00C9A20
:1088B000C00C9AD00C198689A8990C9A200C9A3071
:1088C0000C9A400C9A500C9A600C9A700C9A800C7E
:1088D000096A6C9B200154990C9A400C12109A4220
:1088E000849A4084890C9A400C9A500C9A700C9A85
:1088F00060489A90189A80189A50789A600C9A70EA
:108900000C9A800C9A900C9AA00C9AB00C9AC00CFD
:108910009AD00C096A6C9B700254990C9A900C12B4
:10892000A08A4054990C9AC00C9AD00C213A520C4F
:108930005A10085A20085A30085A40085A50085A03
:1089400060085A70085A80087A90285AB228490854
:108950005A70085A80085A90085AA0085AB0085A03
:10896000C0085AD0085AE0085AF008114A01085ABB
:1089700010085A20085A30085A40085A50085A60BD
:10898000085A70085A80085A90085AA0085AB00825
:108990005AC0086AD0404B0344404B0346404B0347
:1089A00048404B03504059085AB008111C2D310162
:1089B0000111320A290463DD3714010102326429EE
:1089C000046B3936147A03147A7128120423F401E3
:1089D000290473813826480440011405FF78563471
:1089E0001201FF01FF01FF01FF01FF01FF01FF0174
:1089F000FF01FF01FF01FF01FF01FF01FF01FF0177
:108A0000FF01FF01FF01FF01FF01FF01FF01FF0166
:108A1000FF01FF01FF01FF01FF01FF01FF01FF0156
:108A2000FF016D23011105FF7856341201FF01FF8C
:108A300001FF01FF01FF01FF01FF01FF016D5A016D
:108A40000413C0192420B95813143B24207559135A
:108A5000A0441C20315A1C221305FF785634120101
:108A6000FF01FF015B0000000000000000000000AB
:108A700000000000000000000000000000000000F6
:04000005000001A94D
:00000001FF
